:020000040000FA
:06080000D2EF38F01200F7
:0608080081EF32F0120046
:06082A0006003C72000014
:1008300075030000040000001A7200009602000018
:1008400022000000F27100006E020000280000008B
:10085000F0710000FD01000002000000EE710000D8
:10086000FE00000002000000DE7100002D03000009
:040870001000000074
:0C0874000B01006B0A0E005D26E2005133
:10088000220DF3CF01FBF4CF02FB000E01270C0E6B
:100890000223DFEC0CF0EF6A34EC0EF0EF9034EC56
:1008A0000EF0EF8234EC0EF0EF8434EC0EF0EF98A3
:1008B00034EC0EF0EF96DFEC0CF0EFEC0DF0DFEC2B
:1008C0000CF003EC0EF0002BD7D70101496B040E9E
:1008D0004A6F4B6B4C6B4D6B4E6B12000B01006BF8
:1008E0000A0E005D36E20051220DF3CF01FBF4CF7A
:1008F00002FB000E01270C0E0223CEEC0CF0EF5091
:10090000000925E1CEEC0CF0010EEF6ECEEC0CF000
:100910000B0E4FC1EBFF0C0E50C1EBFFCEEC0CF0F9
:100920000D0EEB6A0E0EEB6ACEEC0CF0FFEC0DF048
:1009300046EC0EF0EF8046EC0EF0EF96CEEC0CF0AD
:10094000EFEC0DF046EC0EF0EF8200511200002BA0
:10095000C7D7FE0C0B016F6B6C6B0A0E6C5D14E25B
:100960006C51220DF3CF6DFBF4CF6EFB000E6D27A3
:100970000C0E6E2385EC0CF0EF50000903E1010E24
:100980006F6F02D06C2BE9D76F5101E1FE0C0101B2
:10099000492B000E4A2385EC0CF00B0E49C1EBFFEE
:1009A0000C0E4AC1EBFF880ED8804955130E4A55EC
:1009B00003E2496B040E4A6F85EC0CF0A1EC0DF0DC
:1009C000EF9085EC0CF00D0E53C1EBFF0E0E54C1F1
:1009D000EBFF4B2B000E4C234D234E2307EC0EF068
:1009E00043EC0DF085EC0CF0180E6DEC0CF067ECA0
:1009F0000DF00A0EE66EE66A51C1E6FF52C1E6FF4F
:100A000085EC0CF08FEC0CF0F9EC0CF00101020E0F
:100A10007E6F85EC0CF0F3EC0DF007EC0EF0E9ECDA
:100A20000CF085EC0CF0F7EC0DF085EC0CF0FBEC29
:100A30000DF085EC0CF0D8EC0CF085EC0CF0030E0E
:100A4000EF6E07EC0EF093EC0DF085EC0CF0F2EC91
:100A50000CF00B016C51120001015551A8EC0CF087
:100A6000EF50040801E0000C010C01015651220D69
:100A7000F3CF81FBF4CF82FB000E0B0181270C0E1C
:100A80008223E4EC0CF0EF50040806E081CB88F1FF
:100A900082CB89F1CCEF0AF056C160F14CD9F9EC68
:100AA0000CF00101110E7E6FE4EC0CF0F3EC0DF094
:100AB000E4EC0CF037EC0EF0E9EC0CF0E4EC0CF0AC
:100AC000F7EC0DF0E4EC0CF0FBEC0DF0E4EC0CF0CA
:100AD000D8EC0CF0E4EC0CF037EC0EF093EC0DF0ED
:100AE000E4EC0CF0050EEF6E120001015751220DDF
:100AF000F3CF83FBF4CF84FB000E0B0183270C0E96
:100B000084238AEC0CF09DEC0DF001E1000C8AECE2
:100B10000CF023EC0EF0020B01E1000C8AEC0CF05F
:100B2000100E6DEC0CF0EECF80F1EDCF81F18AEC80
:100B30000CF00F0EEB5001017F6F0101100E7E6F64
:100B4000F3EC0DF08AEC0CF037EC0EF0E9EC0CF065
:100B50008AEC0CF0F7EC0DF08AEC0CF0FBEC0DF0ED
:100B60008AEC0CF0D8EC0CF08AEC0CF0100EC8EC0F
:100B70000DF0126A136A8AEC0CF037EC0EF010508C
:100B8000EE261150EE221250EE221350EE2255ECBA
:100B90000EF0EF9255EC0EF0EF988AEC0CF022EC90
:100BA0000DF08AEC0CF0EFEC0DF055EC0EF0EF824E
:100BB000010C0A0E0101585D13E25851A8EC0CF02B
:100BC0000F0E6DEC0CF0EF50FF0802E134EF18F05F
:100BD0005851A8EC0CF023EC0EF0020B02E0010CD3
:100BE000000E120001015951220DF3CF81FBF4CF09
:100BF00082FB000E0B0181270C0E8223D3EC0CF03C
:100C00009DEC0DF014E1D3EC0CF00F0E1BC0EBFFCC
:100C1000D3EC0CF0EB500201596F6CEC19F0D3ECF3
:100C20000CF04CEC0DF0D3EC0CF07BEC0DF0D3ECB5
:100C30000CF026EC0EF001E3000CD3EC0CF0A1EC70
:100C40000DF0EF885AC150F242EC18F0D3EC0CF0E2
:100C5000100E6DEC0CF0EE2AEF22D3EC0CF026EC2B
:100C60000EF003E359C157F140DF010C01015B5164
:100C7000220DF3CF6CFBF4CF6DFB000E0B016C2744
:100C80000C0E6D23B7EC0CF09DEC0DF014E1B7ECFD
:100C90000CF00F0E1BC0EBFFB7EC0CF0EB50020199
:100CA000596F6CEC19F0B7EC0CF04CEC0DF0B7ECA4
:100CB0000CF07BEC0DF0B7EC0CF026EC0EF001E341
:100CC000000C0DEC0EF0EE24106E5F51EE20116E54
:100CD000CA0ED8801054030E11540EE2B7EC0CF07B
:100CE000100E6DEC0CF0EECF5EF1EFCF5FF1CA0E9F
:100CF000D8805E57030E5F57B7EC0CF0A1EC0DF0F7
:100D0000EF885EC153F25FC154F25CC151F25DC124
:100D100052F264EC18F00DEC0EF0EE265F51ED226D
:100D2000B7EC0CF026EC0EF003E35BC157F1DDDE0F
:100D300001015E51120001016051220DF3CF00FB51
:100D4000F4CF01FB000E0B0100270C0E012300CB9A
:100D5000E9FF01CBEAFF52EC0EF001E1000C7AEC66
:100D600019F000CBE9FF01CBEAFFA1EC0DF0EF9603
:100D7000010C01016151220DF3CF20FBF4CF21FBC7
:100D8000000E0B0120270C0E212318EC0DF052EC65
:100D90000EF02BE018EC0DF023EC0EF0040B08E045
:100DA000280E1DEC0DF018EC0DF0A1EC0DF0EF94F9
:100DB00018EC0DF04CEC0EF0EE50ED1008E17AEC72
:100DC00019F018EC0DF0A1EC0DF0EF96000C18ECFA
:100DD0000DF04CEC0EF0EE06EF5AE2EC18F062C1AA
:100DE000E9FF63C1EAFFEF6E010C000C01016451E1
:100DF000220DF3CF02FBF4CF03FB000E0B01022701
:100E00000C0E0323FFEC0CF052EC0EF03AE0FFEC7A
:100E10000CF023EC0EF0040B08E0280E1DEC0DF096
:100E2000FFEC0CF0A1EC0DF0EF94FFEC0CF0120EC7
:100E3000C8EC0DF001016751105C6851115808E2CF
:100E4000FFEC0CF04CEC0EF0EECF67F1EDCF68F15B
:100E5000FFEC0CF04CEC0EF0EE50ED1008E17AECEB
:100E600019F0FFEC0CF0A1EC0DF0EF960AD067C181
:100E700057F268C158F265C155F266C156F220EFCB
:100E800019F0F36AF46A12000A0E0101695D07E2C3
:100E90006951A8EC0CF052EC0EF002E0010C000ECF
:100EA00012000B01736B6C6B0A0E6C5D01E3D4D006
:100EB0006C51220DF3CF6DFBF4CF6EFB000E6D274E
:100EC0000C0E6E237BEC0CF052EC0EF001E0C1D066
:100ED0007BEC0CF023EC0EF0100B01E0BAD07BECB5
:100EE0000CF0EF50000901E1B4D07BEC0CF0EF50B6
:100EF000010807E17BEC0CF023EC0EF0010B01E0A4
:100F0000A8D07BEC0CF01D0E6DEC0CF00301EE5044
:100F1000645D106EEE506559116E7BEC0CF01F0E87
:100F20006DEC0CF071EC0DF01050125C1150135878
:100F300001E38FD034EC18F0000901E112007BECE2
:100F40000CF0F2EC0CF07BEC0CF01F0E6DEC0CF0E6
:100F5000EE2AEF227BEC0CF01C0E6DEC0CF0EF2A6D
:100F60007BEC0CF0EF50060A27E0010A25E0020AAC
:100F70001CE00F0A1AE00E0A10E0060A05E0010A5A
:100F800028E10B01020E24D013EC0EF0106E030EBC
:100F9000105C16E20B01120E1BD00B01110E736FC9
:100FA0007BEC0CF0050EEF6E14D013EC0EF0030882
:100FB00007E30B01010E0CD013EC0EF0030806E260
:100FC0006DCB88F16ECB89F1E7DA03D00B01100EFF
:100FD000736F0B01735100083CE2100E735D11E05A
:100FE0007BEC0CF037EC0EF0EFCF6FFBEE2AEFCF7F
:100FF00070FBEE22EFCF71FBEE22EFCF72FBEF2200
:101000000CD07BEC0CF037EC0EF0EECF6FFBEECF9C
:1010100070FBEECF71FBEFCF72FBF9EC0CF073CBF2
:101020007EF17BEC0CF0F3EC0DF06FCB76F170CB36
:1010300077F171CB78F172CB79F17BEC0CF0F7ECB6
:101040000DF07BEC0CF0FBEC0DF07BEC0CF0D8EC35
:101050000CF00B016C2B28D71200140E0201576FF5
:10106000586B02016C0E556F0B0E566F20EC19F089
:1010700001016C0E866F0B0E876F59DA6AC1E9FFAA
:101080006BC1EAFF4FEC0EF0EECF80FBEECF81FBA1
:10109000EECF82FBEFCF83FB98EC0DF0EFCF84FB1C
:1010A000010E6DEC0CF0EFCF85FB98EC0DF0020E0D
:1010B0006DEC0CF0EFCF86FB98EC0DF0030E6DECB1
:1010C0000CF0EFCF87FB0B01886B060E896F6EC1AA
:1010D0008AFB6FC18BFB6EC1D8F26FC1D9F274EC81
:1010E00028F0F3CF8AFBF4CF8BFB0C0E0201E06FEC
:1010F000E16B0201800EDE6F0B0EDF6FA8EC28F0B3
:10110000F3CF8DFBF4CF8EFB0B018D1F8E1F240EB2
:101110001DEC0DF08DCB50F242EC18F08ECB50F25E
:1011200042EC18F0140E1DEC0DF06EC1E2F26FC12E
:10113000E3F204EC29F0F3CF8DFBF4CF8EFB0B012F
:101140007C51F31802E17D518E1903E07AEC19F01D
:10115000010C55EC0DF0106E116A140E105E000EAD
:10116000115A10C08FFB1050106E116AE850010127
:101170006E5D6E6F11506F596F6F140E6E5F000EC3
:101180006F5B0B0155EC0DF00201696F6A6B140E79
:101190006927000E6A2317EC1BF06AC184F16BC14A
:1011A00085F101016C0E826F0B0E836F3ED90B012E
:1011B0008C6FFE0E8C5D11E26EC18FF16FC190F1EC
:1011C00001016C0E8D6F0B0E8E6F6AC18BF16BC1BE
:1011D0008CF18CCB8AF106DA010C7AEC19F0FF0E57
:1011E0000B018C5D37E101016E510B017427010188
:1011F0006F510B017523000E762377237951020B73
:1012000003E17951010B05E0742B000E7523762361
:101210007723EFDB0101040E7E6F70CB7AF171CB87
:101220007BF172CB7CF173CB7DF174CB76F175CB16
:1012300077F176CB78F177CB79F16CCB74F16DCB1C
:1012400075F16ECB72F16FCB73F16AC170F16BC146
:1012500071F101D8010C72C148FB73C149FB74C123
:101260004AFB75C14BFB76C14CFB77C14DFB78C186
:101270004EFB79C14FFB7AC150FB7BC151FB7CC156
:1012800052FB7DC153FB0B015491549354955497D9
:101290007EC155FB8DEC19F0F3CF56FBF4CF57FB15
:1012A0000B01000EF35C040EF45804E3566B040EBD
:1012B000576F0DD0360ED8805655000E575505E2A3
:1012C000360E565F000E575B02D0566B576B586B4D
:1012D000596B5A6B5B6B0101480E866F0B0E876F63
:1012E00026D9140E01018027000E81237EA30ED083
:1012F000040E8027000E81230B01020E5C6F040E8A
:101300005D6F5E6F5F6B5499548B03D00B015489F2
:10131000549B548D549FB8C260FBB9C261FBBAC2E2
:1013200062FBBBC263FB70C1E9FF71C1EAFF4FEC16
:101330000EF0EECF64FBEECF65FBEECF66FBEFCF9A
:1013400067FB686B060E696F80C16AFB81C16BFB2E
:1013500080C1D8F281C1D9F274EC28F0F3CF6AFBD6
:10136000F4CF6BFB0C0E0201E06FE16B0201600E2B
:10137000DE6F0B0EDF6FA8EC28F0F3CF58FBF4CF35
:1013800059FB0B01581F591F58CB46FB59CB47FB44
:10139000FF0E01017F5D02E11BC07FF1140E41DBF6
:1013A00080C157F381C158F30301060E566F70C117
:1013B00054F371C155F3DFEC2AF0140E0201536FA0
:1013C000546B0201480E516F0B0E526F64EC18F013
:1013D00001017EA30BD0040E0201536F546B020176
:1013E0005C0E516F0B0E526F64EC18F0140E19DB8B
:1013F00080C1E2F281C1E3F204EC29F0F3CF46FBB5
:10140000F4CF47FB240E0DDB47CB50F242EC18F033
:1014100046CB50F242EC18F002016C6B6D6B7FC151
:101420006BF22AEC1BF0C9EF1AF00B01FE0E036FF2
:10143000026B0A0E025D4AE202511BDB84DAEF50B6
:10144000000941E080DA0B0EA3DB50DB020E45DA27
:1014500048DB00011250101836E11350111833E127
:1014600072DAEF50010802E102CB03FB6CDA0D0ED9
:101470008FDB3CDB36DB1250101825E113501118BE
:1014800022E184C1E9FF85C1EAFF4FEC0EF0EECF07
:1014900014F0EECF15F0EECF16F0EFCF17F053DAD1
:1014A000EE524FEC0EF0EE5014180DE1EE50151800
:1014B0000AE1EE50161807E1EE50171804E103E1B7
:1014C0000B01025112000B01022BB3D70351D1DAE9
:1014D000FE0E035D27E037DAEF50010823E10A0E24
:1014E000E66EE66A84C1E6FF85C1E6FF2CDA17DA0C
:1014F0001250FCDA020E4CDB26DA0B0E10C0EBFFAA
:101500000C0E11C0EBFFF2DA2DDA1DDAFADA1BDA73
:1015100018DBEF9618DA63DB16DA13DBEF820B01C8
:1015200003511200FE0E035D01E1FF0CFE0CDED93B
:10153000EFCF07FBA2DBE552E750EF6ED7D92BDBED
:10154000020E35DB020E09DB020E2BDB020EA1DBE5
:10155000040E09DB040E30DB080E05DB080E2CDB65
:101560000E0E25DB0E0EF9DA0E0E1BDB0E0E91DBD6
:10157000100E1DDB100EF1DA100E13DB100E89DBDE
:10158000120E15DB120EE9DA120E0BDB85DB010EF3
:10159000A4D907CBEFFF1200D1D9CFDA06E0CED91C
:1015A00051DACCD91CDB84DBEF82C8D928DBC6D961
:1015B0000D0EEB6A0E0EEB6AC1D974DB02E07AEC19
:1015C00019F076DBEF96BAD91EDB72DBEF98B6D94D
:1015D0003ADB010B04E0B2D9010EEF6E1200AED976
:1015E000EF6A12000B01A26B01018A51220DF3CFA9
:1015F000A0FBF4CFA1FB000E0B01A0270C0EA12332
:10160000A8DAEECF98FBEECF99FBEECF9AFBEFCFA7
:101610009BFBA6DAEECF9CFBEECF9DFBEECF9EFBB5
:10162000EFCF9FFB6DD9040E58D948DA01018F51D5
:101630000B019027010190510B019123000E922381
:10164000932308DBC4DADFDAE5DA01083AE17AEC61
:1016500019F001014B2B000E4C234D234E2380DA51
:1016600012DA0B01902B91239223932303DBF2DAFE
:1016700077DA59DA69DA020B14E00A0EE66EE66AE6
:101680008BC1E6FF8CC1E6FF2CD949D9125038D95D
:1016900069D927D936DA0B01120EA26F22D9020EB0
:1016A000DCD0040EA26F90CB94FB91CB95FB92CB38
:1016B00096FB93CB97FB24D910D900DA12D99FDA85
:1016C000D9D042DA040B04E07AEC19F088EF0DF07F
:1016D00017D9080E02D99451EE1801E0C9D09551DE
:1016E000EE1801E0C5D09651EE1801E0C1D0975137
:1016F000EE1801E0BDD001E0BBD08CDA02080AE1AF
:10170000C2DA01E1B5D0B6DA62DA040EEF6EA0D922
:101710002CE3AED07FDA03082AE116DA020B01E1EE
:10172000A7D0902B000E912392239323A3DAABDA58
:1017300006E0100EA26FD5D8040EEF6E13D0120E75
:10174000A26FCFD8020EEF6E942B000E9523962336
:10175000972306DA94CBEEFF95CBEEFF96CBEEFF08
:1017600097CBEEFF75D901E383D061DA83D0C8D877
:10177000040EB3D8EECF10F0EECF11F0B2D9E9D904
:101780001050EE1808E11150EE1805E11250EE1855
:1017900002E11350EE1802E07AEF19F06BDA3ADA50
:1017A000040842E170DA09E09CD8C7D906E099D86C
:1017B00049D997D814DA7FDAEF82C6D9010B15E040
:1017C0000B01110EA26FCCD9EFCF94FBEE2AEFCF15
:1017D00095FBEE22EFCF96FBEE22EFCF97FBEF22A9
:1017E000B8D912D97ED80A0EEF6E32D941E279D833
:1017F00059DA05E11CDA0B01100EA26F3BD00B0188
:10180000A26BAED99CCBEEFF9DCBEEFF9ECBEEFF45
:101810009FCBEEFF9ED998CBEEFF99CBEEFF9ACBF4
:10182000EEFF9BCBEEFF24D0F5D90A0805E17AEC58
:1018300019F029DA1FE01AD0EDD9050810E17AEC89
:1018400019F082D9010B16E00B01100EA26F81D99D
:10185000DBD819DA0BE145D8060EEF6E0BD0DAD9DA
:10186000060808E17AEC19F00EDA04E051D902D04A
:101870007AEC19F00B01A25100081EE2BAD8A2CBF3
:101880007EF190CB7AF191CB7BF192CB7CF193CB33
:101890007DF194CB76F195CB77F196CB78F197CB20
:1018A00079F12ED8DCD82CD8020E17D8DDD88BC110
:1018B00070F18CC171F1CFDC120001019151220D48
:1018C000F3CF10F0F4CF11F0000E10260C0E112201
:1018D00010C0F3FF11C0F4FF1200E926000EEA2247
:1018E0001200A0CBE9FFA1CBEAFF120086C1E9FFFD
:1018F00087C1EAFF12006DCBE9FF6ECBEAFF120051
:101900008DC1E9FF8EC1EAFF12006DCBE9FF6ECBFE
:10191000EAFF120083CBE9FF84CBEAFF1200EE520C
:10192000E9CF10F0EACF11F0E9CFE6FFEACFE6FF0A
:10193000A9EC34F0126E060EE15E120088C1E9FFD8
:1019400089C1EAFF120000CBE9FF01CBEAFF1200D8
:10195000220DF3CFE9FFF4CFEAFF000EE9260C0ECB
:10196000EA221200EECF10F0EFCF11F012006CCB94
:10197000E9FF6DCBEAFF1200EECF7AF1EECF7BF1FB
:10198000EECF7CF1EFCF7DF1120090CBEEFF91CB4B
:10199000EEFF92CBEEFF93CBEEFF120001CBE9FFFF
:1019A00002CBEAFF120081CBE9FF82CBEAFF1200F3
:1019B000EE52E9CF70F1EACF71F12BEF09F001CBD4
:1019C000E9FF02CBEAFF120081CBE9FF82CBEAFFFD
:1019D0001200EECF76F1EECF77F1EECF78F1EFCFC8
:1019E00079F112001D0E64C3EBFF1E0E65C3EBFF01
:1019F00012000101806B816B01017F69120002CB33
:101A0000E9FF03CBEAFF1200EF2AEECF90FBEF22B3
:101A1000EECF91FBEF22EECF92FBEF22EFCF93FBC5
:101A2000120002016C6F6D6B7FC16BF22AEF1BF02D
:101A300020CBE9FF21CBEAFF12000201696F6A6B3C
:101A400017EF1BF00F0EEB5002015A6F72EF19F0F7
:101A50000101000ED8808F55000E90551200EECF78
:101A600074F1EDCF75F11200EECF72F1EDCF73F19D
:101A70001200220DF3CF00FBF4CF01FB000E002774
:101A80000C0E012312004BC1EEFF4CC1EEFF4DC105
:101A9000EEFF4EC1EEFF1200100EEB6A110EEB6A64
:101AA000280E02016C6F6D6B12007851F00BE8424A
:101AB000E842E842E842040DF3501200EECF90FBFA
:101AC000EECF91FBEECF92FBEFCF93FB1200EE6ACD
:101AD000EE6AEE6AEE6A1200CA0E105C030E11582E
:101AE0001200EECF12F0EFCF13F0120082C1E9FF27
:101AF00083C1EAFF12000F0EEB5002016B6F2AEF59
:101B00001BF00D0E10C0EBFF0E0E11C0EBFF12000C
:101B1000A0CB88F1A1CB89F1CCEF0AF0700EEE6E6C
:101B2000170EED6E1200EE2AEE22EE22EE221200C9
:101B30006CC1E9FF6DC1EAFF12000F0EEB50FF0808
:101B40001200210E6DEF0CF0DBDE0D0EC6DEEF5045
:101B50001200C7DE180E6DEF0CF0BFDE3DEF0EF089
:101B6000C0DE37EF0EF0B9DEEECFDAF2EECFDBF209
:101B7000EECFDCF2EFCFDDF279EC28F004C010F00C
:101B800005C011F006C012F007C013F076EF0CF09C
:101B9000A4DEB2EF0CF0010EA0DE07CBEFFF76EF74
:101BA0000CF09BDEE552E750EF6E76EF0CF095DE21
:101BB000EFCF07FB76EF0CF090DE04C0EEFF11C014
:101BC000EEFF12C0EEFF13C0EEFF76EF0CF089DEE1
:101BD0001C0E83DEEF6A85DE05DF71EF0CF00F0E61
:101BE0007CDEEF681200180E78DEBCEF0CF00D0EF4
:101BF00074DE2FEF0DF00B0E70DE34EF0DF0EE52B1
:101C00004ED867EF0DF01F0E68DE8EEF0DF07DDE13
:101C100037EF0EF066DEEF501200A9DE100E5DDE2B
:101C200001015E51120067DE1C0EEB50120043D81A
:101C3000EF8657DE120E8FC1EBFF130E90C1EBFF44
:101C40003AD8EF8412007DDFEF501200100EA0DFB3
:101C50006CEF0DF085DFEECF94FBEECF95FBEECF72
:101C600096FBEFCF97FB1200AADEA1EF0DF0140E4A
:101C70006DEF0CF06EDFC5EF0CF0010E2EDEEF50B5
:101C8000E66E76EF0CF060DF100B120087DEA1EF3E
:101C90000DF023DECBEF0DF0120E6DEF0CF0060E03
:101CA0006DEF0CF0D0DF080B120034DEA1EF0DF069
:0C1CB00045DEA1EF0DF015DEA1EF0DF0F8
:041CBC000D01AA6B01
:101CC00064C3A4FD65C3A5FD0B01036B080E035D92
:101CD00015E2500E01014F6F506B6EEC04F0E66E92
:101CE0000B01E3DBA6EC12F0E0DB020EC0DBEF6AD7
:101CF000DCDB090EBCDBEF6A032BE8D71200ABCDAF
:101D000000FBACCD01FB0B0100CBE9FF01CBEAFFEF
:101D1000002B000E0123EF502E0807E000CBE9FF57
:101D200001CBEAFFEF50EFE10A0C026B0251106E9B
:101D3000116A100E105C000E115814E20251A0DB63
:101D400000CBE6FF01CBE6FFF7EC34F0136E050E97
:101D5000E15E1350000903E10B01025112000B0177
:101D6000022BE4D70A0CBFDB04E0200E0B01005D60
:101D7000FAE00B01016B2B0E0B01005D02E1200E5E
:101D8000006F2F0E005D1FE05C0E005D1CE0200E5A
:101D9000005D1BE03F0E005D18E00D0E005D15E0DC
:101DA0000A0E005D12E00C0E015D0DE2610E005D99
:101DB00005E300517A0802E3200E005F0151012B78
:101DC000AADB00CBEFFF8FDBD6E10B010151A3DBD8
:101DD000EF6A0B0101510CE1E10E106E6F0E93DB07
:101DE000AECDE6FFAFCDE6FF0DEC35F0050EE15EC2
:101DF0003F0E0B01005D01E1010C000C0D01A4512F
:101E00000301645D106E65510D01A555116EE00E64
:101E1000105C2E0E115801E3AA6B0B01876B080EA4
:101E2000875D06E287CBB0FD04D80B01872BF7D77F
:101E300012000D01B0510A0DF3CF7CFBF4CF7DFBF6
:101E4000540E0B017C270D0E7D23010E7A6F0B01C2
:101E50007A5101E182D17A6B05DB64DB0AE17CDB3C
:101E6000EF50020B01E0AFDB77DBEF9479DBEF6A39
:101E70001200F8DA020EEB50070AE9E0010A01E16C
:101E80005CD1030A01E12DD1010AE1E0070ADFE09C
:101E9000010A01E118D1030A01E1D6D0010AD7E114
:101EA000E1DA4DDBD4E00B01010E7A6F64C3A4FDCF
:101EB00065C3A5FD51DBEF6A6ADB0D01B66FAAD9D8
:101EC0000B01796F49DBEF9462DB0101916F5DECEF
:101ED0000CF067DBEE52060ECADA0D01A651EE18C1
:101EE00020E1A751EE181DE1A851EE181AE1A95101
:101EF000EE1817E116E1AA5102E02EDBEF84020E84
:101F0000AA5D02E0000E01D0010E106E25DB10501C
:101F1000010BF36EF346F346F346F70EEF14F3109E
:101F2000EF6E0B01795101E089D00D016C0EAE6F9F
:101F30000B0EAF6F2CDB0D01AD6F15DF0B01806F4A
:101F4000580E6C5D15E108DBEF50040B11E10A0E31
:101F5000E66EE66AEB0E106E6F0ED5DA6C0EE66E6C
:101F60000B0EE66ED4EC34F0136E070EE15E1350E8
:101F70000D016C0EAB6F0B0EAC6FC1DEE66EEADAD4
:101F8000E5DA0B0180510BE001016C0EE96F0B0EDD
:101F9000EA6F7CCBE7F17DCBE8F1A3EC14F018DB22
:101FA000DFDA050EEF6EE6DAD1DA00DB106E060E30
:101FB000105C30E312DB04082DE36C0EE66E0B0EB2
:101FC000E66E26EC35F0E552E552F3CF7BFB05DB00
:101FD000030802E3030E01D0020E0B017B5FFDDA62
:101FE0000B0FE66EB7DAB2DAF8DA4ADA7B51146A26
:101FF0006C0F136E0B0E142213C0E6FF14C0E6FF25
:102000000DEC35F0156E050EE15E1550B3DAE552B4
:10201000E750EF6ECBDAFF0803E1D3DAEF6A06D0C0
:10202000C5DAFE0806E1CDDA030EEF6E99DA050E89
:1020300082D092DAEF8294DA010E7DD0790501E048
:1020400006D78EDA030E77D0B5DA01E100D70B019F
:10205000010E7A6F0D016A0EBB6F6F0EBC6F4EDA08
:102060000D017A0EBB6F6F0EBC6FA7DA73DAEF3417
:10207000EA6AFE0BEA36E96E6E0EE926020EEA22E5
:10208000EECFBBFDEDCFBCFD39DA64DAEFCF10F057
:102090000B0E105C06E30D01890EBB6F6F0EBC6F5B
:1020A0008CDAB0CDB9FDA6D998DA060803E154DA86
:1020B000EF8002D051DAEF90D5D9030ED8D9EF6A6C
:1020C0004FDA020E38D0CED93ADA01E081DA7CCB91
:1020D000B7FD7DCBB8FDDCD8000901E1B8D673DAD5
:1020E00028D068DA01E1B3D66CDAEF34EA6AFE0B85
:1020F000EA36E96E8E0EE926020EEA22EECF7EFB6C
:10210000EDCF7FFB0B017ECBF6FF7FCBF7FF7E2B66
:10211000000E7F230800F5CF7BFBF55005E07BCB5D
:102120005AF1A0D9D1D9EED732DA0101576F75EC47
:1021300005F016DA060EEF6E8AD694D9F3D90AE0C6
:1021400039DA08E024DA0101566F35EC05F008DAD7
:10215000070EEF6E01DAEF947AD61200B4CDE9FFE4
:10216000B5CDEAFFEF040B011E6F1D6BEF6A1F6B0D
:102170001E510D01EA6AB225E96EB351EA22EF6AF7
:102180000B011F5141E101011C0E626F0B0E636FC9
:10219000B1CD61F1B9EC06F0000936E03D0E0B015E
:1021A0001C5D0BE11C6B1E511D5D1EE21D29B4CD93
:1021B000E9FFB5CDEAFFEF6E17D0260E1C5D02E1F8
:1021C000020E0AD0200E1C5D06E00D0E1C5D03E021
:1021D0000A0E1C5D04E1010E1F6F1C6B05D02B0E57
:1021E0001C5D02E1200E1C6F1E511D5D06E2B2CD8A
:1021F000E9FFB3CDEAFF1CCBEFFF0D01B22B000EC0
:10220000B3230B011D2BBCD70B011F5101E1000CA7
:102210001F0512000B01056B040E055D19E2055147
:102220000101626F636B000E62270B0E6323B6CD54
:1022300061F1B9EC06F000090BE00B010551052B2B
:10224000EA6A000FE96E0B0EEA22EF502008E4E183
:102250000B010551EA6A000FE96E0B0EEA22EF6AE4
:10226000470E005D07E1450E015D04E1540E025D7D
:1022700001E1000C500E005D0AE14F0E015D07E127
:10228000530E025D04E1540E035D01E1010C020CEA
:10229000F2D813D901E1A6D00B01856BECD8030E5F
:1022A000EB50040818E0E7D814D9400B0DE1E3D84F
:1022B000010EEB500201386F8FEC27F00B01866F97
:1022C000DAD807D9200B07E0D6D8EF500101576FB5
:1022D00075EC05F0010CCFD8090EC9D8EF50010BF1
:1022E00001E17BD0C8D8030EEB50040A50E0070A86
:1022F00034E0010A1BE0030A0BE0010A6BE1250E42
:10230000865D03E131D9010E26D0010E856F62D0C2
:10231000250E865D03E1010E856F5AD029D9030E83
:10232000A6D886CBEFFF20D9020E15D0610E865DB0
:1023300002E3270E04D0410E865D02E3070E865F9E
:10234000300E865D100DF350E66E12D9020E8FD856
:10235000FDD80AD9030EEF6E3DD0610E865D02E313
:10236000270E04D0410E865D02E3070E865F300E15
:10237000865D106EFDD8020E7AD81050EF12F4D898
:10238000040EEF6E78D873D8EE6AED6A23D001019F
:10239000860EED6F0B0EEE6FB7CDEBF1B8CDECF115
:1023A00040EC15F0F3CF10F0F4CF11F0E1D8F3CFFB
:1023B000EEFF11C0EDFF0B01010E856FD9D8FF0EA6
:1023C000EE1808E1FF0EED1805E1865101E1856B7D
:1023D000CBD8EF6A855101E15BD786CB5AF14BD858
:1023E00073D856D748D8010EEB500201376F68EC0E
:1023F00027F0000C0D01B9510A0DF3CF85FBF4CF86
:1024000086FB540E0B0185270D0E862301010D0E50
:10241000C1D801010A0ECAEF12F00D01BA510A0D1E
:10242000F3CF85FBF4CF86FB540E0B0185270D0EF1
:102430008623BBCDF6FFBCCDF7FF0800F55011E0B9
:102440000D01BBCDF6FFBCCDF7FFBB2B000EBC23AF
:102450000800F5CF5AF185CBE9FF86CBEAFF34D8E7
:10246000E8D712007CCBE9FF7DCBEAFF1200E9261A
:10247000000EEA221200B7CDE9FFB8CDEAFF120044
:10248000040DF3CFF6FFF4CFF7FF2A0EF6266F0EFA
:10249000F722F6CF10F0F7CF11F0126A10C0E6FF66
:1024A00011C0E6FF12C0E6FF120003510A0D79D8F1
:1024B000540EE9260D0EEA221200EF500101586F6A
:1024C000D9EC05F000091200EF500101596FF2EF4D
:1024D00005F0010EEB50080D64D8000EE926020E3F
:1024E000EA22EF5012000101000E626F0B0E636FC3
:1024F000ADCD61F1B9EC06F0000912005ED8B0CDA7
:10250000B9FDFAEF11F0116E126A10C0E6FFE66E27
:1025100012C0E6FF12000D01EA6AAE25E96EAF5166
:10252000EA221200EF500101556F2CEC05F0000972
:102530001200010EEB500201366F60EF27F0EF50F2
:102540000101696F44EC07F000091200E552E75001
:10255000EF6E120036D844D085DF090E37EF12F047
:1025600081DF020E37EF12F086DF030E37EF12F035
:1025700082DF36D00201356B02016C0E336F0B0E19
:10258000346FC3EC26F0E66E6DDFEE5212006ADFA8
:10259000EF5012005A6F85CBE9FF86CBEAFF64EF5C
:1025A00012F0F3CFE9FFF4CFEAFF12005BDF010E78
:1025B000EB50120057DF5DEF12F0B0CDBAFD0DEF1A
:1025C00012F050DF0DD0C8DFEF924CDF99EF12F020
:1025D000DEDF0101606F9BEF06F0BCDFEF50120001
:0625E000040E37EF12F0BB
:0A25E600120053EC17F0040B06E09E
:1025F00053EC17F0080B01E0020C010C000C0B016E
:102600001C6B1D6BE2C1E9FFE3C1EAFFEF506B08F1
:1026100001E080D00B01010E206F0201210EE76F57
:102620000B0EE86F010E0101E2250201E56F000EBD
:102630000101E3210201E66F7EEC29F0000903E1CC
:10264000F36AF46A7FD1E4C1E6FFE5C1E6FF5FEC1F
:102650002FF0E552E552F3CF22FB0B012151110877
:1026600004E2160E0B01215D05E10B011C830B0139
:10267000206B43D00B012151150809E3130E0B0108
:10268000215D04E00B011C8F0B01206B36D00B0188
:1026900021511A0801E331D00B0121511E0801E339
:1026A0002CD00B012151220817E31F0E0B01215DD5
:1026B00004E0210E0B01215D07E10B012251080806
:1026C00002E30B01206B02D00B01206B0B012051A8
:1026D00002E10B011C8511D00B012151300805E3EB
:1026E0000B011C870B01206B08D00B012151320814
:1026F00004E30B011C890B01206B0B01205109E144
:102700000101E65106E022CBA8FF21CBD7F29FECD6
:1027100035F013D1E2C1E9FFE3C1EAFFEFCF10F0DA
:10272000610E105C01E2B5D0E2C1E9FFE3C1EAFF4E
:10273000EF50670801E2ADD0E2C1E9FFE3C1EAFF73
:10274000EF50640807E0E2C1E9FFE3C1EAFFEF50A0
:10275000650803E1F36AF46AF5D0E2C1E9FFE3C179
:10276000EAFFEF509F0F0B011E6F1F6B890E0B01CD
:102770001E270F0E0B011F23010E0101EA6AE2253D
:10278000E96EE351EA22EF5014E10201200EE76FF7
:102790000B0EE86FE4C1E5F2E5C1E6F27EEC29F04C
:1027A000000906E01ECBE9FF1FCBEAFF20CBEFFFBD
:1027B0006FD0010E0101EA6AE225E96EE351EA22D7
:1027C000EF50780833E1020E0101EA6AE225E96E72
:1027D000E351EA22EF50D00F106E010E105204E0C8
:1027E000E846FE0B1006FCE10B01206FE4C1E9FF97
:1027F000E5C1EAFFEF5031080AE10B01201D106E20
:102800001ECBE9FF1FCBEAFF1050EF160ED0E4C13C
:10281000E9FFE5C1EAFFEF50300807E11ECBE9FF11
:102820001FCBEAFF0B012051EF1232D0010E010144
:10283000EA6AE225E96EE351EA22EF50D00F106E0A
:10284000010E105204E0E846FE0B1006FCE10B01FD
:10285000206FE4C1E9FFE5C1EAFFEF5030080AE16B
:102860000B01201D106E1ECBE9FF1FCBEAFF10509D
:10287000EF160ED0E4C1E9FFE5C1EAFFEF503108E1
:1028800007E11ECBE9FF1FCBEAFF0B012051EF123E
:1028900054D0E2C1E9FFE3C1EAFFEF506C082DE13B
:1028A0000101E65129E0010E0101EA6AE225E96E23
:1028B000E351EA22EF50610A11E0030A01E01CD063
:1028C0000201080EED6FE4C1EBF2E5C1ECF23E0E41
:1028D0000201E96FEA6BA3EC29F00ED00201080EA9
:1028E000ED6FE4C1EBF2E5C1ECF2350E0201E96FE8
:1028F000EA6BA3EC29F000D020D0E2C1E9FFE3C1EC
:10290000EAFFEF506D0819E10101E65116E0E4C15C
:10291000E9FFE5C1EAFFEF50720A01E00ED0D3EC07
:102920001AF0FF0E986E966E956E936E000E866E80
:10293000846E836E816EFF0000D01CCBF3FF1DCB35
:10294000F4FF00D012000B01146B156B186BE7C17C
:10295000E0F1E8C1E1F148DE0B01196F140E166FCA
:102960000D01160EB46F0B0EB56F0D01000EB26F98
:102970000B0EB36FB1DAEF500D01B16FAEEC10F08A
:102980000B01176F182B1B6B6C0E005D36E10151AC
:10299000750A2BE0050A45E1010E1B6F3E0E54DA65
:1029A00040E1020E0B01185D3CE1010E1A1539E001
:1029B00093DAEF500101916F5DEC0CF0F3CFE9FF7A
:1029C000F4CFEAFFEE52060E83DAEECFA6FDEECF8D
:1029D000A7FDEECFA8FDEFCFA9FD0D01010EAA6F57
:1029E00043DAEF8441DAEF961CD0010E1B6F350EEF
:1029F0002BDA17E10B011A8114D06D0E005D11E185
:102A000019510FE01651EA6A000FE96E0B0EEA2227
:102A1000EF506F0A06E1010E1B6F0D01AA6B24DA5D
:102A2000EF940B011B5115E119CBE6F11651010191
:102A3000E46FE56B000EE4270B0EE5230101000EA9
:102A4000E26F0B0EE36FDBDDF3500B011413F45058
:102A50001513175101E082D71451020B01E0120047
:102A60001451040B02E0B3EF35F01451080B02E0EF
:102A700002EF36F01451100B02E02EEC36F012008B
:102A8000F7D9020E25DAEFCF01FBF2D9030E20DAD7
:102A9000EFCF02FBEDD9EECF07FBEDCF08FB13DA4A
:102AA000EF6AEBC1E0F1ECC1E1F19EDD0B01096FD2
:102AB000610E025D6DE3025168086AE3006B610E0E
:102AC000025D066F070E0115106E010E105204E034
:102AD000E846FE0B1006FCE10B01056F0651036F83
:102AE000046B920E03270F0E0423D0D909E106517F
:102AF000036F046B890E03270F0E0423008107D098
:102B00000651036F046B800E03270F0E0423F00E93
:102B10000115066FE85004E1B9D934E0310E35D023
:102B2000100E065D0CE1B2D905E10101CA0EF26F8B
:102B3000700E02D10101C70EF26F700EFDD0200E93
:102B4000065D03E1010E001506E0300E065D08E1AA
:102B5000010E001505E0080E011501E1D8D0E8D0FE
:102B6000400E065D08E1010E001505E00101AD0E05
:102B7000F26F700EE1D0500E065D01E0E6D0010E5E
:102B8000001502E0300E01D0310E9DD9EF6EDDD080
:102B90006B0E025D0AE1095101E1D7D001CBD6F2FB
:102BA00095EC35F00101FC6F62D06C0E025D42E1E4
:102BB00009512CE00151040A24E0060A1DE0030A31
:102BC00016E0010A01E0C1D009050CE1350E010152
:102BD000F76FF86BEDC1F5F1EEC1F6F107CBF4F14B
:102BE000C7EF16F00101260EF26F580EA5D00101B5
:102BF000D20EF26F710EA0D00101D80EF26F710EDD
:102C00009BD00101220EF26F580E96D00151030A9B
:102C100008E0030A01E099D001011C0EF26F580E82
:102C20008BD0095102E1300E01D0310E066FE8CF92
:102C3000FCF11DD06E0E025D01E087D0006B0F0E1F
:102C40000115106EC11C0F0B105C01E20083F00E29
:102C50000115066FE85005E10101940EF26F700E48
:102C60006BD0100E065D0BE126D9EFCFFCF1EDC164
:102C7000FAF1EEC1FBF107CBF9F1E8EF16F0200E07
:102C8000065D39E118D9EFCF06FB0751081120E1A5
:102C9000330E03D90750300F0101DA6F2E0EDB6FB0
:102CA000330EFBD803C006FB0B0103500A0DB8D846
:102CB0000101DC6F0A0EF1D807C006FB0B010750BB
:102CC000640DAED80101DD6FDE6B0B01076B086B85
:102CD0000751D5D8F8D8EF6E0751D1D836E007CBD9
:102CE00010F008CB11F0072B000E082307CBF3FFE1
:102CF00008CBF4FF1200300E065D03E1020E001552
:102D000006E1500E065D08E1020E001505E1010125
:102D1000BE0EF26F700E10D0400E065D03E1020E83
:102D2000001506E1600E065D10E1020E00150DE1D2
:102D30000101C30EF26F700EF36FEDC1F0F1EEC141
:102D4000F1F107CBEFF1A8EF16F0F368F468120089
:102D50000101EF51F76AF225F66EF351F7220800F0
:102D6000F550F0C1E9FFF1C1EAFFEF6EF0C1E9FFF4
:102D7000F1C1EAFFEF5003E1F368F4681200EF2BB2
:102D8000EF51116AEFC1F3FF11C0F4FF120001010E
:102D9000F451F7250B010A6F000E0101F821AA6E0C
:102DA0000ACBA9FF3F0EA616A680A850F5C1E9FFE1
:102DB000F6C1EAFFEF6EA85003E1F368F468120071
:102DC000F42BF451116AF4C1F3FF11C0F4FF1200A7
:102DD0000101F95110E1DA0EE66E010EE66EFC51CA
:102DE000E66EE66AD4EC2FF0E552E552E552E55284
:102DF0000101DF6BF96BF95142D8FAC1E9FFFBC160
:102E0000EAFFEF6EF9513BD803E1F368F468120072
:102E1000F92BF951116AF9C1F3FF11C0F4FF120047
:102E2000F3CF10F0F4CF11F0330E0B6E0C6AF3CF2A
:102E300006F0F4CF07F09DEC38F006C010F007C0A4
:102E400011F0300E062412000201F06FF16B0B013D
:102E500016510201EE6FEF6B000EEE270B0EEF2303
:102E6000DBEC29F00009120037D8090E68EF17F0E3
:102E7000EBC1E9FFECC1EAFF040E68EF17F0EA6A64
:102E8000DA0FE96E010EEA22EF50120003CBE9FFE0
:102E900004CBEAFFEF5005151200106E0C6E06CB46
:102EA00007F0C4EF38F0E0C1E9FFE1C1EAFF090E25
:102EB0000FD8EF5012000F0E0115EA6ACA0FE96E23
:102EC000020EEA221200EDC1E9FFEEC1EAFF120094
:102ED000E926000EEA221200E7C1E9FFE8C1EAFF95
:022EE0001200DE
:0E2EE200966A8688988802014A6B4B6B4C6B8F
:102EF0004D6B4E6B4F6B0B01006B0051106E116AE6
:102F0000D890115004E6010E105C000E115814E226
:102F10000051040DF3CF10F0F4CF11F0400E102645
:102F2000000E11220051AFDB10C0EFFF0051ABDBF0
:102F3000EE52EF80002BE1D71B6A0201496933DBB7
:102F4000B7DB02011F0EB1DB0201656F02011F0E2C
:102F5000A9DBAEDB0201210EA0DBAADB0201080E19
:102F6000656F02010E0EC7DB0A0EC5DB0B0ED1DB4F
:102F7000040E656F02010C0ECCDB020E656F0201C0
:102F80000D0E90DBDBDB8EDBB1DB010EC2DB600EF6
:102F9000656F0201020E86DBA9DB030EBADB6569F1
:102FA0000201070EA8DB0F0EB4DB610E76DBBCC29C
:102FB00065F20201010E76DBBDC265F20201020E6E
:102FC00071DBBEC265F20201030E6CDBBFC265F2AB
:102FD0000201040E67DBC0C265F20201050E62DB6E
:102FE000C1C265F20201060E5DDB0B01006B080E2B
:102FF000005D0AE202016569080E0B01002502016D
:1030000051DB0B01002BF3D771DB070E4BDB440EBA
:10301000186E0201220E41DB51DB0D0E7ADBE00E51
:103020003CDB0201C00E656F0201010E64DB040E81
:1030300062DB010E6EDB200E4DEF1BF002010D0E68
:1030400070DB02014A2711504B2302010E0E69DB8F
:1030500002014C2711504D2302010F0E62DB0201C9
:103060004E2711504F231200020149511B5C09E108
:103070000201666BB3DA040B03E10201496964D310
:10308000000C62D325DB86A8FED78D8C6B0E8D6E6F
:10309000836A8D9C86A8FED722DB86A8FED78D8CFE
:1030A000670E8D6E400E836E8D9C86A8FED78D8C2C
:1030B000700E8D6E50C283FF8D9C86A8FED78D8CBE
:1030C000192A000E1A22120002015351541101E173
:1030D0001200010E5315106E116A535110240B018A
:1030E0003E6F0201545111200B013F6F956A670E2C
:1030F0008D6E400E836E8D9C86A8FED78D8C6A0ED9
:103100008D6E3ECB83FF8D9C86A8FED78D8C6B0E7B
:103110008D6E3FCB83FF8D9C86A8FED7E0DA86A814
:10312000FED78D8C02015351192654511A22700E6C
:103130008D6EE4DA86A8FED78D8C53C23CFB54C258
:103140003DFB0B01010E3C5F000E3D5B0B013CCBD8
:1031500010F03DCB11F03C07000E3D5B10501110FC
:1031600030E0080E3C5D000E3D5926E389DA86A862
:10317000FED78D8C85DA86A8FED78D8C81DA86A85D
:10318000FED78D8C7DDA86A8FED78D8C79DA86A85D
:10319000FED78D8C75DA86A8FED78D8C71DA86A85D
:1031A000FED78D8C6DDA86A8FED78D8C080E0B01AC
:1031B0003C5F000E3D5BD5D763DA86A8FED78D8CC9
:1031C000C5D7120085DA86A8FED78D8C6B0E8D6E62
:1031D000836A8D9C86A8FED78D8CFF0E195C1DE13D
:1031E0005F0E1A5C1AE10B013269336932CB67F268
:1031F00033CB68F201DA66DA86A8FED78D8C02013D
:10320000100E53DA0B01316F326B440E336F32CB39
:1032100067F2E8CF68F2F0D910D054DA86A8FED76A
:103220008D8C9568700E8D6E8D9A86A8FED783CF93
:1032300031FB8D8A192A000E1A220B01315112001E
:1032400057C2B5FB58C2B6FB02015751581103E1F2
:10325000F36AF46A1200956A6A0E8D6EB5CB83FF2D
:103260008D9C86A8FED78D8C6B0E8D6EB6CB83FFA2
:103270008D9C86A8FED78D8C25DA86A8FED78D8CEE
:103280000B01B5511926B6511A22600E1A5C02E3E1
:103290001C0E1A5E9568700E8D6E0B01B5CB10F08A
:1032A000B6CB11F0B507000EB65B105011100FE051
:1032B0008D9A86A8FED7020155C2E9FF56C2EAFFE1
:1032C000552B000E562383CFEFFF8D8AE6D757C2CA
:1032D000F3FF58C2F4FF120002015951D4D9EE5243
:1032E000EF90120002015A51CED9EE52EF805AC22D
:1032F0001BF0120018C036FB0B01010E356FE8CF32
:1033000067F218C068F278D95DDF0B01346FE8CF3F
:1033100065F20201030E52EF1BF0FED90B01006FA4
:103320000201200EBAD918500B01005D05E2600EB3
:10333000D8801854002502D01850005D016FE85065
:10334000106E116A1C0ED8801056000E115610C057
:1033500001FB10C003FB026B02CBF3FF10C0F4FFB4
:1033600012000201E00EE5D90B01006F0201200EF0
:1033700094D90B010051040B01E0000C010C5DC25B
:10338000E9FF5EC2EAFFEF68C7D90B01126F0201C5
:10339000200ECFD90B01136FDCD9100B37E00201DF
:1033A000666B1CD9040B0B01176F0201210E75D936
:1033B000020EE66E86EC38F0E55280D90A0E9BD9F3
:1033C0000B0E70D90B01175108E0C3D90A0B02E0AC
:1033D000000E01D0010E0B01176F0201020E656F86
:1033E00002010D0E96D9220E58D912CB18F082DFA9
:1033F000020165690201070E7ED90D0E53D90B013A
:10340000175103E00201260E48D9000C0B0113519D
:10341000125D67E013CB15FB146B14CB67F213CB73
:1034200068F2EAD8120E0201576F586B0201000EC3
:10343000556F0B0E566F04DF0B010051010B4EE070
:10344000400E025D000E035949E3EE0ED88002558E
:10345000050E035543E3600E015D40E20151106E1D
:10346000116AD890115004E6440E105C000E1158F9
:1034700035E310CBD8F211CBD9F274EC28F0F3CFAE
:1034800010FBF4CF11FB060EE66EE66A0A0EE66E3E
:103490000B0EE66E5BC2E9FF5CC2EAFF5BC210F096
:1034A0005CC211F05BC2E6FF5CC2E6FFA9EC34F03F
:1034B000126E060EE15E1250080E0B01115D0BE15B
:1034C000105103E0060E105D06E15DC2E9FF5EC229
:1034D000EAFF10CBEFFF13CB18F0010C12CB18F062
:1034E00009DF000C02010A0E656F0201070EDAD82F
:1034F0001DD9EFCF41FB0B01406B40CB67F241CBB5
:1035000068F27AD8060E0201536F546B5FC251F213
:1035100060C252F2D9DDBCC250F2B4DDBDC250F27D
:10352000B1DDBEC250F2AEDDBFC250F2ABDDC0C2F3
:1035300050F2A8DDC1C250F2A5DD0201615103E1E4
:103540000B01426B03D00B01060E426F0201080E05
:10355000506F98DD42CB50F295DD0E0E02016227CE
:10356000000E63233C0E625D000E635903E23C0EC5
:10357000626F636B62C240FB63C241FB62C265F271
:103580000201050E8FD841CB65F20201060E52EF03
:103590001BF0D4D8BED8240E80D81BC049F2C6D8A0
:1035A000EE52EF8012009568600E8D6E8D8C8D8AC4
:1035B0008D8E966A0A0EE66EDEEC38F0E55278D80B
:1035C0008D9E1200600E020164118D6E65C283FF34
:1035D000956A8D9C86A8FED78D8C12009568600E2A
:1035E000020166118D6E8D9A86A8FED783CF37FBB8
:1035F0008D8A0B013751120067C219F068C21AF0A8
:1036000067C265F20201080E4DD868C265F2020178
:10361000090E52EF1BF00201090E47D80B01016F92
:103620000201080E42D8F36E01CBF4FF120018C05D
:1036300023FB0B01120E226F020169510B0122279D
:1036400002016A510B01232322CB67F223CB68F2DC
:10365000FCEF1AF06BC21BF069D8EFCF0DFB0B012A
:103660000E0E0C6F02016C510B010C2702016D5103
:103670000B010D230CCB67F20DCB68F2FCEF1AF0B7
:1036800002017EEF1BF0E96EEA6AD890E936EA366D
:10369000460EE926020EEA221200656F0201646BF3
:1036A000E2EF1AF0646FE2EF1AF0666FEEEF1AF0D5
:1036B000050EE66E86EC38F0E55212000201656BED
:1036C00002011200600E8D6E0A0E836E8D9C120038
:1036D000956A6A0E8D6E010E836E8D9C12008D8C24
:1036E000600E8D6E120E836E8D9C12000201440ED0
:1036F000656F02011200D6DF5EEF1BF051C2E9FFD9
:1037000052C2EAFF512B000E5223EF50836E8D9C64
:103710001200C8DF020112000201600EBEDFA9EF35
:103720001BF0C3DF106E116AE85012001B5043EF0C
:103730001BF0B3DF0201030E55EF1BF0F7DFEFCFF5
:1037400065F20201040E1200F1DFEE52EF50010BA0
:0A37500012000201070E55EF1BF0F6
:06375A000B01006B020EE2
:10376000005D07E200513BDB00512DDBEF90002BA9
:10377000F6D712000B01000E016F010E026F006BF5
:10378000020E005D43E2DCDA0C0EC7DACADA126A16
:10379000136A105011101210131032E1D1DA0C0E0E
:1037A00029C1EBFF0D0E2AC1EBFF01012B512C119A
:1037B00011E00A0EE66EE66A2BC1E6FF2CC1E6FFB9
:1037C000BFDA01CB10F002CB11F001CBE6FF02CB48
:1037D000E6FFD8DAB5DA0A0E2DC1EBFF0B0E2EC1CB
:1037E000EBFFAEDA0E0EEB6A0F0EEB6AA9DA100EE3
:1037F000EB6A110EEB6A00CB28F10B0100511200AD
:10380000140E0127000E0223002BBAD7FF0C010172
:103810002F51EFEF1EF0020E0101305D04E230C1C6
:1038200028F134EF18F0000C01012851140DF3CFEA
:103830000AFBF4CF0BFB000E0B010A27010E0B2332
:10384000CADAEE50ED1004E190DA94DA8EDA87DA13
:1038500031C150F242EC18F0BEDAEE2AEF22BBDAA8
:10386000C4DA01E346D8010C01012851140DF3CF4D
:103870000AFBF4CF0BFB000E0B010A27010E0B23F2
:10388000A6DAEE50ED1004E151DA74DA4FDA67DAB5
:103890009EDA01013451EE24106E3551EE20116E86
:1038A000D60ED8801054030E11540AE290DAEECFEF
:1038B00034F1EFCF35F1D60ED8803457030E35579B
:1038C00034C153F235C154F232C151F233C152F214
:1038D00064EC18F07CDA01013451EE263551ED220A
:1038E00076DA83DA01E305D834C1F3FF35C1F4FF9A
:1038F000120001012851140DF3CF08FBF4CF09FB8E
:10390000000E0B010827010E092315DA0C0E05DA4B
:1039100040DAF3CF00FBF4CF01FB0DDA0A0EFDD93C
:1039200038DAF3CF02FBF4CF03FB05DA0E0EF5D93C
:10393000EECF04FBEFCF05FB080E0B010427000EB2
:103940000523066B076B140E02016C6F6D6BF3D9C8
:1039500006DA04CB57F305CB58F30301110E566F6B
:10396000EAD908CB54F309CB55F3DFEC2AF004CBAA
:10397000D8F205CBD9F274EC28F0F3CF04FBF4CFE6
:1039800005FB080E0201536F546B0201000E516FCC
:103990000B0E526F64EC18F0C9EC1AF0CCD9120E71
:1039A000BCD9EF68C8D90E0EEB6A0F0EEB6A120095
:1039B000020E0101365D0AE236C128F1FFD9D88036
:1039C000EE54000EED5401E3000C010C000C17DA6C
:1039D00001E1000C2851F7D9EF50010B01E013DA97
:1039E000E2EC18F037C1E9FF38C1EAFFEF6E11DAF7
:1039F000EE06EF5AE3D9EE50ED1002E17AEC19F041
:103A0000010CFDD903E1F36AF46A12002851DBD9F5
:103A1000EF50010B01E0F7D9FCD983D93B51105C81
:103A20003C51115805E2CAD9EECF3BF1EDCF3CF144
:103A30003BC157F23CC158F239C155F23AC156F276
:103A400020EC19F0F3CF00FBF4CF01FBE2D90B011E
:103A50000051EE5E0151ED5AD2D902E17AEC19F033
:103A60003BC1F3FF3CC1F4FF1200C9D902E07AEC7C
:103A700019F0CFD9EE6AED6A1200080E0201576FF5
:103A8000586B0201460E556F0B0E566F20EC19F065
:103A900046CB5DFB47CB46FB5DCB47FB48CB5DFB95
:103AA00049CB48FB5DCB49FB080E106E0B014B5117
:103AB000D880105403E24A055D6F02D04ACB5DFB0B
:103AC000080E4B5D4A6F5DCB4BFB4CCB5DFB4DCB8A
:103AD0004CFB5DCB4DFB3DC1E9FF3EC1EAFF060E4D
:103AE0001CD9EECF4FFBEECF50FBEECF51FBEFCF0B
:103AF00052FB55D9EFCF53FB010E0FD9EFCF54FB3B
:103B00004ED9020E0AD9EFCF55FB49D9030E05D97C
:103B1000EFCF56FB576B110E586F41C159FB42C195
:103B20005AFB41C1D8F242C1D9F274EC28F0F3CF6C
:103B300059FBF4CF5AFB0C0E0201E06FE16B02015E
:103B40004F0EDE6F0B0EDF6FA8EC28F0F3CF5BFBA0
:103B5000F4CF5CFB0B015B1F5C1F1A0EFBD85BCB29
:103B600050F242EC18F05CCB50F242EC18F0140E1C
:103B7000F1D841C1E2F242C1E3F204EC29F0F3CF03
:103B80005BFBF4CF5CFB0B014C51F31816E14D517C
:103B90005C1913E13FC147F140C148F13DC145F116
:103BA0003EC146F10101460E436F0B0E446F1CD817
:103BB0000B014E6FFF0E4E5D03E17AEC19F0010C24
:103BC0004E51A1D8100EA9D84ACBEEFF4BCBEDFF3A
:103BD0004E51F9D8EF80010C0101285194D8E9CF5A
:103BE000F3FFEACFF4FF12000B010169000E026F30
:103BF000010E036F006B020E005D5BE2A6D80C0E97
:103C0000FAD8020E8AD8D5D80001125010184AE10D
:103C10001350111847E199D80A0EEDD8CAD812509E
:103C200010183EE1135011183BE18FD8100E75D8D3
:103C3000EECF14F0EFCF15F0166A176A1450151076
:103C4000161017102DE145C1E9FF46C1EAFF060E27
:103C500064D8EECF10F0EECF11F0ABD876D8060EC8
:103C60005CD8EE50101808E1EE50111805E1EE5046
:103C7000121802E1EE50131810E047C1E9FF48C1E5
:103C8000EAFFE868EE180CE1E868EE1809E1E86878
:103C9000EE1806E1E868EE1803E10B01005112008E
:103CA00000CB01FB0B01140E0227000E0323002B97
:103CB000A2D7FF0E015D24E00151140DF3CF02FBEA
:103CC000F4CF03FB000E0227010E03230A0EE66E5B
:103CD000E66A45C1E6FF46C1E6FF37D802CB10F0E1
:103CE00003CB11F002CBE6FF03CBE6FF4BD85CD849
:103CF00018D82BD80A0E10C0EBFF0B0E11C0EBFF2B
:103D00000B0101511200140DF3CFE9FFF4CFEAFFCC
:103D1000000EE926010EEA221200E926000EEA2230
:103D20001200EECF10F0EFCF11F012000ACBE9FF36
:103D30000BCBEAFF120008CBE9FF09CBEAFF120028
:103D400001CBE9FF02CBEAFF120002CBE9FF03CB74
:103D5000EAFF12000201696F6A6B17EF1BF0120E87
:103D6000EB5002016B6F2AEF1BF00ACBE9FF0BCB84
:103D7000EAFF1200120E1BC0EBFF1C0E02016C6F5B
:103D80006D6B1200A9EC34F0126E060EE15E12505B
:103D90001200EECFD8F2EDCFD9F274EF28F03FC188
:103DA000E9FF40C1EAFF120043C1E9FF44C1EAFF55
:103DB0001200EECF12F0EFCF13F012002851A3DF64
:103DC000100E8DEF1EF09FDF130E8DEF1EF0AEDF95
:103DD0000E0E8DEF1EF0C9DF0E0E8DEF1EF093DF7D
:103DE0000C0E9BDFEE6AED6A12009BDFD60E105CB4
:103DF000030E1158120091DF94DFD4EF1EF009D8A2
:103E0000EE50ED1012002851DEDFEF901C0EAAEFED
:083E10001EF00101DEEF1EF0BF
:083E1800070E0301755D01E1D5
:103E20001200FF0E765D01E0A7DA03017669756B7B
:103E3000786B120003017551060A01E1A2D0030A52
:103E400066E0010A59E0070A46E0010A33E0030A86
:103E500027E0010A01E012000B010E690F691069E9
:103E600011691269136914691569166917690301E3
:103E7000086B096B0A6B0B6B430E01012D6F2E6BE8
:103E800001010E0E2B6F0B0E2C6F440E0101296FDA
:103E90002A6BBAEC1BF00301766F62DA010E756FC4
:103EA00050DA140E105C000E115801E27DD00301AF
:103EB000020E3BD00301085109110A110B1133E125
:103EC00076C330F10BEC1CF000096EE00301010E2B
:103ED0005FDA030E2AD061DA03E30301020E756F85
:103EE00076C336F1D8EC1CF000095EE063D8020816
:103EF0005BE10301040E756F76C330F10BEC1CF02F
:103F0000000952E00301030E43DA050E0ED076C31A
:103F100036F1D8EC1CF000092EE04CD80B01186FDC
:103F2000060E185D04E10301040E756F1200050E04
:103F3000185D26E121DA0301766912DA060E756F43
:103F400008C3B8F209C3B9F20AC3BAF20BC3BBF291
:103F500010C3C2F211C3C3F212C3C4F213C3C5F239
:103F60000CC3C6F20DC3C7F20EC3C8F20FC3C9F229
:103F70007781782B120011DA17E30301020E756FB7
:103F80001200DFD9640E105C000E11580DE3040717
:103F9000000E055B065B075B045105110611071156
:103FA00002E10301756BDCD912000301080E756F85
:103FB000BCEF21F00B01026B03013C0E046F056B9B
:103FC000066B076BB0D9020E0B01005D01E0EBD070
:103FD000016B0F0E015D02E2EFD9FBD70101080E64
:103FE000376F030EABD9090E376F030EA7D90A0E30
:103FF000376F030EA3D90B0E376F030EC6D90B0113
:10400000016B080E015D02E2D7D9FBD7BCC208FBE9
:10401000BDC209FBBEC20AFBBFC20BFBC0C20CFB88
:10402000C1C20DFB016B060E015D0EE27CD90B01D6
:104030000151EA6A080FE96E0B0EEA22EF50005DAB
:1040400001E0D3D0012BEFD7016B0151106E116A43
:10405000D890115004E6CE0E105C000E115802E20A
:10406000ABD9F3D7036B5FD90B010051330A62E080
:10407000CC0A5DE0C90A47E0350A23E0020A0DE0F8
:10408000340A01E07DD04FD90B01000501E0ADD02D
:104090000101020E376F0B0E48D072D901E0A5D096
:1040A0000101100E376F030E49D9110E376F030E41
:1040B00045D9120E376F030E41D9130E376F030E19
:1040C00034D05ED901E291D001010C0E376F030E9E
:1040D00035D90D0E376F030E31D90E0E376F030E23
:1040E0002DD90F0E376F030E50D9040E0B01005F50
:1040F0000B0100510007000952E00101010E376F6A
:104100000B0E43D9F5D73CD970E10101070E376F8B
:104110000B0E14D9060E376F0B0E10D9050E376F24
:104120000B0E0CD9040E376F0B0E2FD938D0010EA1
:10413000036F35D025D959E10101070E376F030E02
:10414000FDD8060E376F030EF9D8050E376F030E34
:10415000F5D8040E376F030E18D9D880080E030166
:104160000455070E0555000E0655000E075517E2BB
:10417000080E045F070E055B000E065B075B0FD0A1
:104180000101000E376F0B0E00D90B010051000723
:10419000000905E00101010E376F0B0EF5D70B0189
:1041A000035101E160D7020E025D09E104CB00F387
:1041B00005CB01F306CB02F307CB03F311D0000EBE
:1041C000E96E030EEA6EEE50041908E1EE5005198F
:1041D00005E1EE50061902E1EE50071901E0026B0D
:1041E00035EC1DF00B010251120035EC1DF0000CF6
:1041F0000101010E9ED8010E9CD8060E9AD8ABD8AC
:10420000120E97D8230E95D8340E93D8560ECBD8CD
:10421000800EC9D8A0D89FD8316B14EC1CF00B01CC
:10422000196B0C0E195D02E2A0D8FBD7BCC231F1AC
:1042300014EC1CF0BDC231F114EC1CF0BEC231F123
:1042400014EC1CF0BFC231F114EC1CF0C0C231F10F
:1042500014EC1CF0C1C231F114EC1CF00B01196B11
:104260001951106E116AD890115004E6CA0E105CF4
:10427000000E115802E279D8F3D70101630E59D824
:10428000820E57D8530E55D8630E53D8350E51D8D9
:10429000010E316F14EC1CF016C331F114EC1CF05C
:1042A0000301160518E0085109110A110B1113E05A
:1042B0000101360E7CD803C331F114EC1CF002C3AB
:1042C00031F114EC1CF001C331F114EC1CF000C30B
:1042D00031F114EC1CF00101370E2BD8020E29D855
:1042E000010E27D8030E316F14EC1CF0030E0301EE
:1042F000165D13E10101320E5AD808C331F114ECF6
:104300001CF009C331F114EC1CF00AC331F114ECB8
:104310001CF00BC331F114EC1CF00101316914ECF9
:104320001CF079EF1CF00101000E376F0B0EC5EF8A
:1043300021F0316F14EC1CF00101120026D80101AC
:104340001200030114510301645D106E65510301F5
:104350001555116E1200316B14EC1CF001011200A6
:1043600064C314F365C315F312000101316B14EC3F
:104370001CF00B01192B120076C32FF107EF1CF074
:10438000D2DF040E0B01005D1200386FE7EF1CF066
:10439000166F2EDFE5DF03011200D3DF900E105CF5
:1043A000FF0E11581200C5DFD6DFABEF21F0C1DFE1
:1043B000040E316F14EF1CF0B6DF0B01012B12005D
:1043C0000001F35101E112000001FD0EF16F640ED6
:1043D000F26FEBEC36F000010D0EF16F630EF26F31
:1043E000EBEC36F0F3C0B4FB0B01B451000814E25F
:1043F000B451070B05E100012E0EED6F8CEC36F089
:1044000027DA02E057D908D0320EE66E86EC38F093
:10441000E5520B01B407E8D72DEF24F03CDAE7D9D9
:10442000010EE926000EEA22E2D9020EE926000E6C
:10443000EA22DDD9030EE926000EEA223EEF24F03F
:104440000B01016B05DAFEE07CEC36F00B01006F2E
:104450000D0E005D17E00A0E005D14E0012B000157
:10446000F6C0E9FFF7C0EAFFF62B000EF72300CBFA
:10447000EFFFF6C0E9FFF7C0EAFFEF6AF851F8076F
:104480000009E0E10B0101511200F9C001FBFAC083
:1044900002FB0B01036BF9C0E9FFFAC0EAFFEFCFA3
:1044A00000FBEF5021E02E0E0B01005D11E1000139
:1044B000F9C0E9FFFAC0EAFFF92B000EFA23EF6A10
:1044C000AFD9032BD1D9F9C001FBFAC002FB07D049
:1044D000300E005D03E30051390801E2000C0001D9
:1044E000F92B000EFA23D7D79BD9BED9030E0B01A7
:1044F000035D01E0000C010CABD9FEE07CEC36F072
:104500000B01006F310E005D05E3390E005D02E224
:1045100000511200390CA1D9300E0001FD5DFF0FD2
:10452000E96EEA6AD890E936EA362D0EE926030EDE
:10453000EA22EECFF1F0EDCFF2F0EBEC36F0000135
:10454000FD51380A01E1B5D00F0A01E1B0D0010AEE
:1045500001E1A1D0030A01E197D0010A54E0070A62
:104560004BE0010A42E0030A01E012000201330EAF
:10457000D66F95EC35F00B01A16F0201340ED66FAA
:1045800095EC35F00B01A26F870EE66E0B0EE66E12
:10459000A1CBE6FFA2CBE6FF87D9870EEF6F0B0E0C
:1045A000F06FDAEC36F029D9000947E0870EE66EA5
:1045B0000B0EE66E5FEC2FF0E552E552F3CFA1FB58
:1045C000F4CFA2FBF3CFA8FF0201330ED76F9FEC0D
:1045D00035F0A2CBA8FF0201340ED76F9FEC35F067
:1045E000A2CBC0F2A1CBC1F212000B01B80E9F6F9B
:1045F000020EA06FA36B0ED00B01C60E9F6F020EB2
:10460000A06F0E0E06D00B01C20E9F6F020EA06FA0
:104610000A0EA36F9FCBF4F0A0CBF5F0FFDEEDD830
:1046200000019B0EFB6F0B0EFC6F0001870EF96FF4
:104630000B0EFA6F2ADF00090BE10001B30EF16FD8
:10464000640EF26FEBEC36F003D9FEE07CEF36F04F
:104650009FCBE9FFA0CBEAFF9BCBEEFF9CCBEEFF0D
:104660009DCBEEFF9ECBEEFF9BCBA8FFEAD89CCB69
:10467000A8FFE7D89DCBA8FFE4D89ECBA8FF0B01ED
:10468000A351A32B020110D00201160ED66F95EC98
:1046900035F0010906D00201160ED66F95EC35F003
:1046A000FE0BA86E0201160ED76F9FEF35F06FEF6D
:1046B00023F012000001460EF16F630EF26FEBEC77
:1046C00036F01ADF0B01B56F390EB55D03E0B5CBDF
:1046D000FDF021DF380E0B01B55DECE112000B019E
:1046E000006B026BF8EC27F064C385FB65C386FBA7
:1046F0000B0185510301645D106E65510B018655F8
:10470000116E320E105C000E115809E364C385FB74
:1047100065C386FB0001150EED6F8CEC36F098D862
:10472000E7E00B01025162E193D8FBE07CEC36F04C
:104730000B01016F0051030A20E0010A1BE0030A8C
:1047400014E0010502E1010E16D0040E015D09E13D
:1047500041EC28F00001060E9BD80B01010E026F00
:10476000E0D70001150E94D8DCD7060E046F036B5A
:10477000020E01D0030E006FD4D70351032BEA6A57
:10478000050FE96E0B0EEA2201CBEFFF0351106E0D
:10479000116A1134C6E210508008000E1154C1E2B3
:1047A000060E046F016B0151106E116AD890115002
:1047B00004E6800E105C000E11580DE20151EA6A09
:1047C000050FE96E0B0EEA22EFCF45F210EC28F050
:1047D0000B01012BE8D70201376B68EC27F004CB03
:1047E000EDF08CEC36F00B01006B9BD7010C46D83A
:1047F00000012E0E4DD84BEF24F00001290E48D8B1
:1048000000013A0E45D80001200E42D80001140ED6
:10481000F86F0001870EF66F0B0EF76F20EF22F096
:1048200001CBE6FF02CBE6FF5FEC2FF0E552E5524D
:10483000F350E66EFBC010F0FCC011F00B01035109
:1048400012000B01A351A32B0201D76F9FEF35F08C
:104850000001EA510001EB5D120000010D0E18D8B5
:1048600000010A0E48EF24F00F011024E96E000E3B
:104870001120EA6EE552E750EF6E1200EF50E66E3F
:10488000E66A12D8000EEF6F0B0EF06FDAEF36F01B
:10489000ED6F8CEF36F0000EE66E0B0EE66EF4C098
:1048A000E9FFF5C0EAFF1200D4EC2FF0E552E55223
:0848B000E552E552000112007F
:0848B800150E01014F6F506B5A
:1048C0006EEC04F00101936F976BC56B926B140E45
:1048D000956F966B120093C155F12CEC05F0000911
:1048E00007E10101C56B070E996F976B926BA6D01C
:1048F00093C169F144EC07F0000934E020DA0101CA
:10490000700E626F0B0E636F93C161F1B9EC06F02C
:1049100000090EE01F0E0101C55DF1E2C551C52B76
:10492000EA6AA40FE96E010EEA2270CBEFFFE7D727
:1049300093C160F19BEC06F00A0E0B01705D26E15D
:104940000101C551EA6AA40FE96E010EEA22EF6A7D
:10495000C56B9BD9C6C1D8F1C7C1D9F15DD90101D9
:10496000996F14D00101975111E0D5510301645D95
:10497000106E65510101D655116E500E105C460E39
:10498000115804E3DCD9020E996F976F010197511A
:10499000020A3EE0070A0DE0040A06E0010A54E1BB
:1049A0009A6BCDD9010E976FBED94EE00101050E6D
:1049B000976FB9D92DE09AC1E9FFEA6AE9BEEA68C2
:1049C000D890E936EA36A20EE926020EEA22EECFA8
:1049D00071FBEDCF72FB0B0171CBF6FF72CBF7FFD2
:1049E000712B000E72230800F5CF70FBF55007E025
:1049F00070CB5AF193C159F1F2EC05F0ECD793C1A9
:104A000057F175EC05F001010B0E9A6F020E976FCE
:104A1000070E0101995D18E099C1D7F116D8000978
:104A20000FE00B0E01019A5D02E0050E04D0020EAC
:104A3000995D02E1010E976F070E996F986B010C5B
:104A40000B0E01019A5DB3E1010C0101D751050A7A
:104A500051E0060A4DE0070A34E0060A30E0030A96
:104A600018E0010A51E192819293010E9A6F090EAA
:104A7000E66EE66AC8C1E6FFC9C1E6FF9B0EE66EB8
:104A8000010EE66E34EC35F0106E060EE15E10504D
:104A9000010C92A112D0C8C16FF3C9C170F3030118
:104AA0009B0E6D6F010E6E6F5FEC33F0000904E03A
:104AB00001019283020E29D00101060E26D087EF54
:104AC00025F0D0C1E6FFD1C1E6FF5FEC2FF0E55243
:104AD000E552F3CF96F1D2C1E6FFD3C1E6FF5FEC1A
:104AE0002FF0E552E552F3CF95F101010A0E0DD0FA
:104AF000B0EF25F00A0E9A6FFE0E945D07E094C1A8
:104B000056F135EC05F0010C050E9A6F010C010110
:104B10009851030A18E0020A0FE0010A20E1020E90
:104B2000985D02E141EC28F0FE0E0101945D06E083
:104B300010D90101010E05D0FCD811E10101030ECD
:104B40009A6F986F000CEFD80AE093C155F12CECE6
:104B500005F0000904E093C156F135EC05F0000CB6
:104B600001019851020A2EE0030A21E0010A53E1F3
:104B700092B302D0060E4DD0070E9A6F95C153F135
:104B800096C154F19351220DF3CFE9FFF4CFEAFF20
:104B9000000EE9260C0EEA22EE52E9CF51F1EACFDF
:104BA00052F1AAEC04F00101946F010E09D0C1D8B2
:104BB00032E0020131A12FD0F8EC27F00101020E02
:104BC000986F000C94C169F144EC07F000091AE0F9
:104BD000B6D80101730E626F0B0E636F94C161F161
:104BE000B9EC06F0000905E073CB45F210EC28F0B3
:104BF000F0D70201376B68EC27F094C160F19BECB1
:104C000006F0000C96D807E1A4D80101FE0E946FBF
:104C1000090E9A6F010C000C0B01006B060EE76E7B
:104C20000019E8AE02D0E73402D0E750005D2CE274
:104C3000040EE66EE66A00CBE9FFEA6AE9BEEA68BE
:104C4000D890E936EA36960EE926020EEA22EECF31
:104C500010F0EFCF11F0126A10C0E6FF11C0E6FFAE
:104C600012C0E6FFD8C1E6FFD9C1E6FF8AEC34F0F6
:104C7000136E070EE15E1350000903E10B010051B2
:104C800012000B01002BCAD7060C0B01036BA40EFC
:104C9000006F010E016F58D8EF50200804E1002B7F
:104CA000000E0123F8D700CBC6F101CBC7F10101FB
:104CB000010ED46F49D8EFCF02FBEF5033E00B0168
:104CC0000351010A16E0010A29E1200E025D03E00A
:104CD0002C0E025D05E138D8EF6A010E036F1ED07D
:104CE0000D0E025D03E00A0E025D18E12DD8EF6A99
:104CF00015D0200E025D12E00101D451D42BE96ED3
:104D0000EA6AD890E936EA36C60EE926010EEA22AA
:104D100000CBEEFF01CBEDFF0B01036B002B000E70
:104D20000123C8D7120093C158F1D9EC05F000094E
:104D3000120094C155F12CEC05F00009120064C377
:104D4000D5F165C3D6F1120000CBE9FF01CBEAFF34
:0E4D5000120041EC28F094C156F135EF05F049
:024D5E00020150
:104D6000306B010E316F0301180E3D6F8AEC33F08A
:104D70000B01006B060E005D05E2005191D9EF6A50
:104D8000002BF8D7010C0B01FE0E026F020131A1BE
:104D9000FE0C0B01016B060E015D0AE2015180D988
:104DA000EF50010B03E101CB02FB02D0012BF3D743
:104DB000FE0E025D01E1FE0C450E036F046B056BF8
:104DC00033C2E9FF34C2EAFFEF5001E1FF0C33C206
:104DD000E6FF34C2E6FF62EC35F0E552E552F3CF70
:104DE00033F2F4CF34F203CB42F304CB43F367D96D
:104DF00004E00B01FE0E026F5ED014EC34F00B01E8
:104E0000006F00AF02D0026956D0016B0C0E015D3D
:104E100021E214EC34F00B01006F01510201EA6A47
:104E20003325E96E3451EA22EF500B01005D06E0B4
:104E3000120E0327000E042305230CD0005108E1B5
:104E40000B01012B0C0E015D05E214EC34F0F8D7D8
:104E5000012BDCD70C0E015D2BE10251080DF3CFC5
:104E600006FBF4CF07FB000E0627020E072333D9FB
:104E7000010EEF6E30D9EB6A020EEB6A14EC34F0DF
:104E8000E66E29D9030E03D9030E2AD9010EFFD8E5
:104E9000030E26D9020EFBD8060EF9D8060E20D92D
:104EA000010E1ED9E552E750EF6E0201302B03D000
:104EB0001EEC34F098D71EEC34F00B0102511200B6
:104EC00036C237F205D802013651EAD8EF6A12002D
:104ED00002013751080DF3CFAFFBF4CFB0FB000E4A
:104EE0000B01AF27020EB023F1D8EF50020B03E005
:104EF0001EEC34F00DD0EAD8EF50040B09E00AECB8
:104F000034F00301A00E4B6F59EC34F00009F9E1C5
:104F1000F90EDCD8E850EF160201319312000201BD
:104F20003851080DF3CF01FBF4CF02FB000E0B014B
:104F30000127020E02239F0E106EBCD8E850EF1618
:104F4000B9D8EF50010B25E0B5D8EF50020B24E1A2
:104F5000020131B31ED0AED8EE52EECF13F0EFCF38
:104F600014F0156AA7D8030EBBD8EE501324106EA8
:104F7000EE501420116EEE501520126E10C042F348
:104F800011C043F39CD805E195D8EF82020131832B
:104F900003D090D8EF8A000C14EC34F00B01006FB2
:104FA00089D8EE52EE2A000EED22EECF10F0EDCFB2
:104FB00011F080D8060E94D8EECF12F0EFCF13F098
:104FC00000011250101805E11350111802E172D8B7
:104FD000EF8C0B0100511200010C010C12001200A9
:104FE000F36AF46A1200056A066A076A1200000C86
:104FF000020131A1000C0B01AF6B060EAF5D08E2A0
:10500000AF514ED8EF50010B01E0000CAF2BF5D79C
:105010000201010E006F400E036F046B056B010C63
:105020000B01000EB16F020EB26F020100A506D097
:10503000400E325D03E30201376B4ADF020100B527
:1050400015D031A302D0008B000C03C23FF304C281
:1050500040F30301A00E3E6F93EC33F0000905E12D
:10506000020100853183326B01D0000C45C244F34C
:10507000F6EC33F00201322B032B000E0423052340
:10508000010C0201376B24DF0201006B010C28D8F0
:10509000E552E750EF6E14EC34F0E66E6BEF28F05B
:1050A000080DF3CFE9FFF4CFEAFF000EE926020E68
:1050B000EA22120001CBE9FF02CBEAFF1200030152
:1050C000A00E416FC9EC33F000091200AFCBE9FF2D
:1050D000B0CBEAFF120006CBE9FF07CBEAFF1200D4
:0850E000E926000EEA2212008D
:0850E800D9C2F3FFD8C2F4FFA6
:1050F0001200DAC201FBDBC202FBDCC203FBDDC231
:1051000004FB0B01010E056F0B0E066F05CBE9FFCB
:10511000EA6E030E9AD9EF50E66E030E90D900CBDB
:10512000EFFF84D9020E91D9010E85D9EF50E66EBA
:105130007DD9020E84D9010E7ED900CBEFFF01CBC1
:1051400004F002CB05F003CB06F004CB07F012000D
:105150000B01406B416B426B436BDEC23EFBDFC217
:105160003FFBE0C23CFBE1C23DFBD8903D333C330A
:105170003CCB10F03DCB11F03C07000E3D5B1050D6
:10518000111018E03ECBE9FF3FCBEAFF020E3E27AD
:10519000000E3F23EECF10F0EFCF11F000011050C2
:1051A0000B014027000111500B014123000E422347
:1051B0004323DED70201E051010B0EE03ECBE9FFB5
:1051C0003FCBEAFFEFCF10F0000110500B0140275A
:1051D000000E4123422343230B014251431109E0B6
:1051E00040514225406F41514321416F426B436B17
:1051F000F3D740CB10F041CB11F0101E111E10C0A0
:10520000F3FF11C0F4FF12000B01010E006F016BE0
:10521000026B0201E251E3114EE0400EE25D000E2E
:10522000E35904E3400E106E116A04D0E2C210F09C
:10523000E3C211F010C005FB0B0110500201576FC3
:10524000586B0201060E556F0B0E566F20EC19F0CD
:105250000B010551106E116A10500201E25F1150EE
:10526000E35B0B01046B0551045DD3E20451EA6A70
:10527000060FE96E0B0EEA22EFCF03FB00510AE1A5
:1052800003510125016F0351015D0DE2022B0BE17A
:10529000012B09D003510225026F0351025D03E285
:1052A000012B01E1022B005102E0000E01D0010EA2
:1052B000006F042BD8D70B01021D026F011DF36E86
:1052C00002CBF4FF12000201E451390805E3300E6D
:1052D000E45D02E3300E0FD0E451460805E3410ED1
:1052E000E45D02E3370E07D0E451660806E3610E81
:1052F000E45D03E3570EE45D1200FF0C010E0201B2
:10530000EA6AE525E96EE651EA22EFCFE4F2DBDF57
:105310000B01236FE5C2E9FFE6C2EAFFEFCFE4F23B
:10532000D2DF0B01246FFF0E235D03E0FF0E245D2F
:1053300001E1000C2439F00B2311E7C2E9FFE8C2B8
:10534000EAFFEF6E010C0B01236BA6B2FED72F0E06
:10535000A616A6840201EBC2E9FFECC2EAFFEB2B22
:10536000000EEC23EF50A86E0B01232B0201ED5130
:105370000B01D880235501E2A86AEAC210F0116A35
:105380001050AA6E0201E9C210F0EAC211F0E92B36
:10539000000EEA231050A96E550EA76EAA0EA76E36
:1053A000A6820000A6B2FED7A850D4E1A6940B01B5
:1053B000235100D01200F1C210F01050AA6EF0C2BA
:1053C000A9FF3F0EA6160201EEC2E9FFEFC2EAFFF7
:1053D000EE2B000EEF23EFCF1CFBA680A8500B0195
:1053E0001C5D01E0010C1C5101E1000CA92AEBE15C
:1053F000AA2AE9D7F2C202FBF3C203FB0B01006B3E
:10540000016B0201F4510B01005D0201F5510B012A
:1054100001590BE202CBE9FF03CBEAFF022B000E9E
:105420000323EF6A002B0123ECD7120005CBE9FF21
:1054300006CBEAFF1200E926000EEA221200FBDF8B
:10544000E552E750EF6E16EF2AF0F5DFEFCF00FBE5
:0454500016EF2AF039
:0C545400140E0201576F586B0201080E85
:10546000556F0B0E566F20EC19F0F00E0B0108155E
:10547000400801E0A1D00F0E0815040DF350106E86
:10548000116A140E105E000E115A10C01CFB105051
:10549000140801E291D01C5100080BE21C510201DA
:1054A000576F586B02011D0E556F0B0E566F20EC97
:1054B00019F012CB00FB13CB01FB0B01126B136B2A
:1054C000140E16D9080EDE6F0B0EDF6FA8EC28F055
:1054D000F3CF04FBF4CF05FB0B01041F051F1C5188
:1054E000000810E21C5104D91D0EDE6F0B0EDF6F99
:1054F000A8EC28F0F3CF06FBF4CF07FB0B01061F47
:10550000071F02D0066B076B040EF2D8040EDE6F85
:105510000B0EDF6FA8EC28F0F3CF02FBF4CF03FBF8
:105520000301080E596F0B0E5A6FB5D80B010251CB
:10553000001942E1035101193FE1F00E081540083E
:105540003BE103014C514D110CE04CC3E9FF4DC34D
:10555000EAFF18CBEEFF19CBEEFF1ACBEEFF1BCB09
:10556000EEFF4EC3E9FF4FC3EAFF060EDBD814CBB4
:10557000EEFF15CBEEFF16CBEEFF17CBEEFF50C3C1
:10558000E9FF51C3EAFF11CBEFFF0B011C51126E73
:10559000136A12500A5D106E13500B59116E140EDF
:1055A000105E000E115A52C3E9FF53C3EAFF10C048
:1055B000EEFF11C0EDFF010C7AEC19F0000C0B01AD
:1055C000450E286F296B140E030157250B012A6F16
:1055D000000E030158210B012B6F0101FD2B000E62
:1055E000FE23FDC12CFBFEC12DFB0B012E6B400EDB
:1055F0002F6F640E306F56C331FB326B336BB8C202
:1056000034FBB9C235FBBAC236FBBBC237FB54C34D
:10561000E9FF55C3EAFF060E85D8EECF38FBEECF83
:1056200039FBEECF3AFBEFCF3BFB0301280E596F5E
:105630000B0E5A6F30D8140E5BD8280EDE6F0B0E8F
:10564000DF6FA8EC28F0F3CF32FBF4CF33FB140E5E
:10565000030157250201626F000E03015821020168
:10566000636F0201616B54C3E9FF55C3EAFF54C382
:105670005FF255C360F272EC1AF0140E0201536F20
:10568000546B0201280E516F0B0E526F64EC18F030
:10569000F36AF46A120027D8020E35D8020E38D801
:1056A000020E2BD8020E39D8040E2DD8040E30D895
:1056B000040E23D8040E31D8060E25D8060E28D89D
:1056C000060E1BD8060E29D80A0E1DD80A0E20D8A1
:1056D0000A0E13D80A0E03D83CCBEFFF120022D8D3
:1056E000010E92EF2BF059C3E9FF5AC3EAFF1200F3
:1056F0000201E06FE16B0201120014D8E552E7509D
:10570000EF6E73EF2BF00ED8EFCF3CFB73EF2BF067
:10571000E6DFEF50E66E73EF2BF0E1DF3CCBEFFFFF
:0C57200073EF2BF0E926000EEA221200C5
:04572C004854545039
:105730002F312E3020353033200D0A0D0A5365727B
:105740007669636520556E617661696C61626C652E
:105750000D0A000D0A0D0A00485454502F312E3006
:1057600020323030204F4B0D0A436F6E74656E74DB
:105770002D747970653A2000485454502F312E30E2
:1057800020343034204E6F7420666F756E640D0ABD
:105790000D0A4E6F7420666F756E642E0D0A0061DF
:1057A0007564696F2F782D77617665006170706C14
:1057B00069636174696F6E2F6A6176612D617263CE
:1057C0006869766500696D6167652F6A7065670055
:1057D000696D6167652F67696600746578742F6A03
:1057E00061766173637269707400746578742F6395
:1057F0007373006170706C69636174696F6E2F6A96
:105800006176612D766D00746578742F68746D6CA7
:1058100000746578742F706C61696E0047756573EC
:105820007400596573005375706572205573657205
:10583000000D0A4E6F772072756E6E696E6720617B
:1058400070706C69636174696F6E2E2E2E000D0A84
:10585000526561647920746F20646F776E6C6F613C
:10586000642046696C652053797374656D20496DB9
:10587000616765202D2055736520586D6F64656DD7
:105880002070726F746F636F6C2E0D0A000D0A44E6
:10589000484350202620495020476C65616E696E50
:1058A000672064697361626C65642E0D0A000D0ADD
:1058B00044484350202620495020476C65616E695A
:1058C0006E6720656E61626C65642E0D0A000D0ABC
:1058D00044656661756C74205375626E6574204D05
:1058E00061736B2028000D0A44656661756C742035
:1058F00047617465776179204164647265737320D0
:1059000028000D0A44656661756C74204950204179
:105910006464726573732028000D0A5365726961AF
:105920006C204E756D626572202800323030206F19
:105930006B0D0A00323236205472616E73666572E6
:1059400020436F6D706C6574650D0A00313235202F
:10595000446F6E652E0D0A00313530205472616E31
:105960007366657272696E6720646174612E2E2E93
:105970000D0A00353330204C6F67696E20726571F7
:1059800075697265640D0A00353032204E6F7420DF
:10599000696D706C656D656E7465640D0A003530F7
:1059A00030200D0A00323231204279650D0A003272
:1059B0003330204C6F6767656420696E0D0A0033D1
:1059C00033312050617373776F7264207265717523
:1059D000697265640D0A0032323020526561647963
:1059E0000D0A0041424F5200504F52540053544F41
:1059F000520051554954005041535300555345529C
:015A000000A5
:0E5A02001C0E0201576F586B0201000E556F0B
:105A10000B0E566F20EC19F07AEC19F00301000E12
:105A2000626F0B0E636FF5D80B01010E001912E1C6
:105A3000015110E10451106E116A060E10180AE1AE
:105A4000115008E10551126E136A040E121801E19B
:105A5000135001E0000C020E061905E1075103E1A5
:105A600006D9EF6A0DD0010E061906E1075104E1CF
:105A7000010EFDD8EF6E04D0020EF9D8EF6E000CC7
:105A80000201B8510B01185D2EE10201B9510B0161
:105A9000195D29E10201BA510B011A5D24E10201ED
:105AA000BB510B011B5D1FE15BC3E9FF5CC3EAFF58
:105AB00008CBEEFF09CBEEFF0ACBEEFF0BCBEEFFE0
:105AC0000CCBEEFF0DCBEEFF5BC3E9FF5CC3EAFF3F
:105AD000060ED7D80ECBEEFF0FCBEEFF10CBEEFFAE
:105AE00011CBEEFF010C000C010E0B01006F016BDE
:105AF000026B080E036F060E046F040E056F0301A0
:105B000061050BE1010E0B01066F076B126913694A
:105B1000146915691669176914D0020E0B01066F16
:105B2000076B5FC3E9FF60C3EAFFEECF12FBEECF66
:105B300013FBEECF14FBEECF15FBEECF16FBEFCF32
:105B400017FBBCC208FBBDC209FBBEC20AFBBFC239
:105B50000BFBC0C20CFBC1C20DFBB8C20EFBB9C22D
:105B60000FFBBAC210FBBBC211FB7AD8EF500E1963
:105B70000201C2151BE174D8010E83D8EF500B014E
:105B80000F190201C31512E16BD8020E7AD8EF503B
:105B90000B0110190201C41509E162D8030E71D876
:105BA000EF500B0111190201C51509E0C6C218FB1F
:105BB000C7C219FBC8C21AFBC9C21BFB09D050D807
:105BC000EECF18FBEECF19FBEECF1AFBEFCF1BFB8E
:105BD0000301000E626F0B0E636F1BD81C0E0201D7
:105BE000626F636B0201060E616F0201120E5F6F3E
:105BF0000B0E606F72EC1AF01C0E0201536F546BA7
:105C00000201000E516F0B0E526F64EC18F0C9EFD9
:105C10001AF032D819D8F3CFEEFF11C0EDFF2CD80F
:105C2000020E2FD811D8020EF3CFEBFF030E11C0D6
:105C3000EBFF22D8060E25D807D8060EF3CFEBFFD0
:105C4000070E11C0EBFF1200EECFD8F2EDCFD9F264
:105C500074EC28F0F3CF10F0F4CF11F03CEF2EF0FD
:105C60005FC3E9FF60C3EAFF060E41EF2EF05DC39C
:105C7000E9FF5EC3EAFF120062C3E9FF63C3EAFF04
:0A5C80001200E926000EEA221200CD
:065C8A000D01BD6BBE819F
:105C900071EC17F0FDEC36F0ADEC1BF03AEF04F0D0
:105CA0000B01010EB46F0B01B45101E1FDD0B46BD7
:105CB0000D01BD51040A01E1D7D0070A01E1A1D0CD
:105CC000050A01E187D0010A72E0050A3FE0070AF0
:105CD00036E0050A02E0010AE6E10201B30E5D6F5B
:105CE0000B0E5E6F0201BF0E5B6F0D0E5C6FBFECA3
:105CF00019F0000915E10201160ED66F95EC35F08A
:105D0000010BD1E0B1EC19F00009CDE10201B86B53
:105D1000B96BBA6BBB6B0D01BE810CEC1FF0C3D726
:105D20000B01010EB46FB35103E10D01020E39D026
:105D3000060EB35D01E095D00D01050E32D00B01CA
:105D4000B46B0AEC37F00009AEE0ABD00301C90E2A
:105D5000526F0D0E536F0301B30E506F0B0E516F48
:105D60000301BF0E4E6F0D0E4F6F0301AF0E4C6F50
:105D70000B0E4D6F2AEC2AF0000916E00B01010E04
:105D8000B46FB30503E10D01030E0BD0060EB35D36
:105D900003E10D01060E05D0110EB35D04E10D0106
:105DA000070EBD6F80D7B46B7AEC19F07AD0C9CDED
:105DB00041F1CACD42F10101AF0E3F6F0B0E406FB2
:105DC0000101BF0E3D6F0D0E3E6F3DEC1DF0000951
:105DD00015E012D0C9CD6EF1CACD6FF10101AF0E41
:105DE0006C6F0B0E6D6F0101BF0E6A6F0D0E6B6F46
:105DF0002DEC08F0000902E00D01BD6B0B01B46B46
:105E000052D7BD6B290ED880C955000ECA5529E35B
:105E10000301ED0E1F6F0D0E206F0301EB0E1D6FC2
:105E20000D0E1E6F0301C90E1B6F0D0E1C6F0301BB
:105E3000CB0E196F0D0E1A6F0301B30E176F0B0EF9
:105E4000186F6EEC30F000090AE0080E0B01B35D2C
:105E500006E1010EB46F0D01040EBD6F02D00D01FD
:105E6000BD6B7AEC19F01FD734EC18F0000901E192
:105E70001AD7EDCD29F3EECD2AF3EBCD27F3ECCDF8
:105E800028F3C9CD26F30301CB0E246F0D0E256F29
:105E90000301236B0301BF0E216F0D0E226FE8EC8F
:105EA00030F00D01BD6BFFD651EC07F01AEC1FF07E
:0E5EB000030177A102D00D01BE911EEF18F084
:025EBE00FF0ED5
:105EC000E3CFEAFFE552FF0EE3CFE9FFE552E66AD2
:105ED000E66AD9CFE6FFDACFE6FFFC0EE124D96E01
:105EE000FF0EE220DA6EE66AE66AE66A200EEF5CF2
:105EF00006E0090EEF5C03E0EF6603D03FD0EE5002
:105F0000F5D72D0EEF5C03E1FF0EE32A03D02B0E35
:105F1000EF5C01E1EE502F0EEF6424D03A0EEF60FB
:105F200021D0D890F90EE336FA0EE336FD0EDECF1F
:105F3000E3FFFE0EDDCFE3FFD890F90EE336FA0E55
:105F4000E336D890F90EE336FA0EE336FD0EE35051
:105F5000DE26FE0EE350DD22300EEE5CDE26000E65
:105F6000DD22D9D7FF0EE3CFE8FFE85207E0F90EB4
:105F7000E31EE32AFA0ED8B4E306E31EE552E55227
:105F8000E552FF0EE3CFDAFFE552FF0EE3CFD9FF74
:105F9000E552E1CFE9FFE2CFEAFFED52ED52EECF5D
:105FA000F3FFEFCFF4FF1200D9CFE6FFDACFE6FF21
:105FB000FA0EE3CFD9FFFB0EE3CFDAFFFD0EE3527B
:105FC00009E72D0EDE6EFC0EE31EE32AFD0ED8B4AB
:105FD000E306E31EE652E652E652FD0EE124E76ECA
:105FE000FF0EE220E46EE652F70EE3CFE6FFF70E77
:105FF000E3CFE6FF44EC30F0F90EE124E96EFF0E4A
:10600000E220EA6E34EC30F00AE131EC30F009E1E4
:1060100034EC30F008E131EC30F007E108D03FEC2F
:1060200030F03AEC30F03FEC30F03AEC30F03FEC4E
:1060300030F0DE6AF90EE126FF0EE222FF0EE3CF1A
:10604000DAFFE552FF0EE3CFD9FFE552FC0EE12463
:10605000E96EFF0EE220EA6EEECFF3FFEFCFF4FF22
:106060001200EF380F0B1200EF500F0B02E1EE524F
:10607000D8841200EF380F0B300FDE6E1200EE5096
:106080000F0B300FDE6E1200FC0EE3CFE9FFFD0EAA
:10609000E3CFEAFF100EE66EEE6AEE6AEF6AD89082
:1060A000FD0EE336FE0EE336ED36ED36EF36FF0E2F
:1060B000E30609E065EC30F0EE5265EC30F0EE52AC
:1060C00065EC30F0EDD7E56E1200030EEF24E8B674
:0C60D000EF6E300EEF24E8BEEF6E000C07
:0460DC00080E0201A7
:1060E000576F586B0201000E556F0B0E566F20EC68
:1060F00019F002CB2EFB03CB2FFB0B01026B036BC2
:10610000080E0201E06FE16B0201000EDE6F0B0E64
:10611000DF6FA8EC28F0F3CF28FBF4CF29FB0B01AD
:10612000281F291F080E106ED9D8E850EF5ED6D868
:10613000EF500201576F586B19C355F21AC356F24C
:1061400020EC19F0CBD8EF500201E06FE16B19C3DE
:10615000DEF21AC3DFF2A8EC28F0F3CF2AFBF4CF6B
:106160002BFB0B012A1F2B1F040E0201E06FE16BBA
:106170000201280EDE6F0B0EDF6FA8EC28F0F3CFC4
:106180002CFBF4CF2DFB0301000E2B6F0B0E2C6F9D
:106190007AD817C3E9FF18C3EAFF00CBEFFF1DC38E
:1061A000E9FF1EC3EAFF04CBEEFF05CBEDFF1FC3E3
:1061B000E9FF20C3EAFF06CBEEFF07CBEDFF0B01A3
:1061C0002E512C1902E12F512D1901E0000C010C68
:1061D0000B01016B23C300FB026B036B27C304FBA2
:1061E00028C305FB29C306FB2AC307FB030126516D
:1061F000E66EE66A24C3E6FF25C3E6FF080EE66EF8
:106200000B0EE66EA9EC34F0106E060EE15E105037
:106210000301000E2B6F0B0E2C6F35D8080E0301F7
:1062200026250201E06FE16B000EE1230201000E62
:10623000DE6F0B0EDF6FA8EC28F0F3CF02FBF4CF7C
:1062400003FB080E030126250301576F586B000E50
:1062500058230301010E566F21C354F322C355F393
:10626000DFEC2AF0080E030126250201536F546B60
:10627000000E54230201000E516F0B0E526F64EC9E
:1062800018F0C9EF1AF02FD8040E15D8040EF3CF6A
:10629000EBFF050E1FD8060E0ED8060EF3CFEBFF50
:1062A000070E18D8020E07D8020EF3CFEBFF030E2D
:1062B00011C0EBFF1200E926000EEA22EECFD8F261
:1062C000EDCFD9F274EC28F0F3CF10F0F4CF11F049
:1062D00073EF31F011C0EBFF73EF31F01BC3E9FF37
:1062E0001CC3EAFF12002BC3E9FF2CC3EAFF120014
:1062F0004D6F6474726F6E6978205443502F49500B
:1063000020537461636B2056332E3033000D0A50D6
:106310007265737320616E79206B657920666F7288
:1063200020436F6E66696775726174696F6E206D68
:10633000656E752E00444843502F476C65616E6949
:106340006E672E2E2E000D0A0D0A0D4D78576562D0
:10635000537276722044656D6F204170706C696372
:106360006174696F6E2076312E3020284D6F647411
:10637000726F6E6978205443502F495020537461D6
:10638000636B2056332E30332C2046656220323228
:106390002032303036290D0A0D0A09313A2043687F
:1063A000616E676520426F61726420736572696116
:1063B0006C206E756D6265722E0D0A09323A2043AB
:1063C00068616E67652064656661756C742049500C
:1063D00020616464726573732E0D0A09333A204399
:1063E00068616E67652064656661756C74206761BD
:1063F000746577617920616464726573732E0D0A28
:1064000009343A204368616E67652064656661758A
:106410006C74207375626E6574206D61736B2E0DE4
:106420000A09353A20456E61626C65204448435044
:10643000202620495020476C65616E696E672E0DDD
:106440000A09363A2044697361626C652044484306
:1064500050202620495020476C65616E696E672E7A
:106460000D0A09373A20446F776E6C6F61642046DD
:10647000696C652053797374656D20496D6167653A
:106480002E0D0A09383A2053617665202620517571
:1064900069742E0D0A0D0A456E7465722061206DB7
:1064A000656E752063686F6963652028312D382912
:1064B0003A20000D0A496E76616C696420696E703D
:1064C0007574207265636569766564202D20496E58
:1064D0007075742069676E6F7265642E0D0A507254
:1064E00065737320616E79206B657920746F20630A
:1064F0006F6E74696E75652E2E2E0D0A001B5B3251
:026500004A004F
:0E650200DACFE4FFE2CFDAFFE9CFE4FFEACF21
:10651000E4FFF6CFE4FFF7CFE4FFF5CFE4FFF3CFDE
:10652000E4FFF4CFE4FFFACFE4FF00EE00F0100E3A
:10653000E80403E3EECFE4FFFBD700EE10F0080E13
:10654000E80403E3EECFE4FFFBD7E652F2A414D055
:106550009E0ED76E580ED66E0301642B000E652377
:106560006623672303016A0706E1640E6A6F03016D
:10657000682B000E6923F2949E50200B05E09D507D
:10658000200B02E04FEC36F09E50100B05E09D50C2
:10659000100B02E065EC36F0E55200EE17F0080E45
:1065A000E80403E3E5CFEDFFFBD700EE0FF0100E9C
:1065B000E80403E3E5CFEDFFFBD7E5CFFAFFE5CF36
:1065C000F4FFE5CFF3FFE5CFF5FFE5CFF7FFE5CF2C
:1065D000F6FFE5CFEAFFE5CFE9FFE5CFDAFF1100EF
:1065E00088D8B3EC38F0AFEC26F0F3EC12F03BECCB
:1065F00036F077EC35F0B3EC35F044EC36F002ECE5
:1066000036F019EC36F02EEC36F00201140ED66F8F
:1066100095EC35F00001F36FE0EC21F045EC2EF045
:106620005EEC0EF05CEC24F00201160ED66F95ECD9
:1066300035F0010B06E10001010EFE6F0301070EAC
:10664000756F0201150ED66F95EC35F0020B0CE05C
:106650000001FF510301645D106E320E105C04E313
:1066600064C3FFF0939C8A7C50EC2EF0FEEC0EF09D
:106670006BEC24F008D80001FE510301785DE1E0E5
:1066800078C3FEF0DED703016C2B0C0E6C5D01E3CA
:106690006C6BC11C0F0B6C5D0FE2C30EC2166C510C
:1066A000040DF350C212C280C282C2B2FED70301EF
:1066B0002AD8C4CFEFFF120026D8EF6A1200350E99
:1066C0000201F06FF16B6DC3EEF26EC3EFF2DBEC23
:1066D00029F000090DE13E0E0201F06FF16B6FC36E
:1066E000EEF270C3EFF2DBEC29F0000901E1010CDE
:1066F000000C040ED36ED3A6FED7D382F18ED56ADA
:10670000F28EF28C12006C51EA6ACA0FE96E020E28
:04671000EA22120067
:0C6714003DC373F30301726B0301080E18
:10672000716F6BEF38F03FC3AFFB40C3B0FBC75096
:10673000040B01E0010EE5D8FAE1C580C5B0FED733
:10674000A1B6010C3EC374F3E1D801E0010CC750BF
:10675000040B01E0010ED5D8FAE1C5BC19D0B0CBCD
:1067600074F3D4D801E0010CC750040B01E0010E12
:10677000C8D8FAE1AFCB74F3C9D801E0010CC75017
:10678000040B01E0010EBDD8FAE1C5AC000C020C0F
:10679000020C42C33FF343C340F341C33EF3C3DFA4
:1067A0000B01086FE85005E178D80B01086FE8503D
:1067B00002E008511200C750040B01E0010EA1D8FD
:1067C000FAE1C580C5B0FED7A1B6010C030141298D
:1067D0000301746F9BD801E0010CC750040B01E06A
:1067E000010E8FD8FAE1C5AC000C020CC750040BA7
:1067F00001E0010E86D8FAE144C374F387D801E0C2
:10680000010CC750040B01E0010E7BD8FAE1C5ACC6
:10681000000C020CC750040B01E0010E72D8FAE123
:10682000C584C5B4FED7000C7AEC38F0C5B6FED7E7
:10683000C59AC588C5B8FED7C95012007AEC38F0A1
:10684000C5B6FED7C58AC588C5B8FED7C584C5B448
:10685000FED7000C46C342F347C343F345C341F39D
:1068600098DF0B01006FE85016E103014A514A0717
:1068700000090EE0D9DFE66E030148C3E9FF49C312
:10688000EAFF482B000E4923E552E750EF6EEDD7A3
:10689000D5DF0B01006F00511200C750040B01E05F
:1068A000010E2FD8FAE1C584C5B4FED7A1B6010CFC
:1068B000000CC750040B01E0010E23D8FAE1C5809B
:1068C000C5B0FED7A1B6010C4BC374F31FD801E0CD
:1068D000010CC750040B01E0010E13D8FAE1A1B678
:1068E000010CC5BC03D00B01B36B03D00B01040E2C
:1068F000B36FC584C5B4FED7A1B6010C0B01B3516B
:106900001200106E1F0EC514101012007FEC38F02C
:046910000009120068
:0C691400FB0EE3CFF6FFFC0EE3CFF7FF15
:10692000FD0EE3CFF8FFFE0EE3CFE9FFFF0EE3CF4E
:10693000EAFFF90EE35003E1FA0EE35009E0F90E25
:10694000E30602E2FA0EE3060900F550EE5CF1E020
:106950001200D9CFE6FFDACFE6FFFA0EE3CFD9FF78
:10696000FB0EE3CFDAFFFC0EE3CFE9FFFD0EE3CF32
:10697000EAFFE9CFF3FFEACFF4FFF80EE35003E1BB
:10698000F90EE35008E0F80EE30602E2F90EE30622
:10699000DECFEEFFF2D7FF0EE3CFDAFFE552FF0EB8
:1069A000E3CFD9FFE5521200FB0EE3CFF6FFFC0E5A
:1069B000E3CFF7FFFD0EE3CFF8FFFE0EE3CFE9FFD5
:1069C000FF0EE3CFEAFFE9CFF3FFEACFF4FFF90EC2
:1069D000E35003E1FA0EE35009E0F90EE30602E2A8
:1069E000FA0EE3060900F5CFEEFFF1D71200FB0E19
:1069F000E3CFF6FFFC0EE3CFF7FFFD0EE3CFF8FF8A
:106A0000FE0EE3CFE9FFFF0EE3CFEAFF0900F550EA
:106A1000EF5C02E1EE66FAD71200FB0EE3CFF6FF61
:106A2000FC0EE3CFF7FFFD0EE3CFF8FFFE0EE3CF42
:106A3000E9FFFF0EE3CFEAFFE9CFF3FFEACFF4FF70
:106A40000900F5CFEFFFEE66FBD71200FE0EE3CF95
:106A5000E9FFFF0EE3CFEAFFF36AF46AEE5203E0C8
:106A6000F34AF42AFBD71200D9CFE6FFDACFE6FFCC
:106A7000FA0EE3CFD9FFFB0EE3CFDAFFFC0EE3CF34
:106A8000E9FFFD0EE3CFEAFFE9CFF3FFEACFF4FF22
:106A9000F80EE35003E1F90EE3500BE0F80EE306C5
:106AA00002E2F90EE306DECFEFFFEE66F1D7DD522C
:106AB000EFD7FF0EE3CFDAFFE552FF0EE3CFD9FFAA
:106AC000E5521200FE0EE3CFE9FFFF0EE3CFEAFF2F
:106AD000E9CFF3FFEACFF4FF610EEF5C05E67B0E32
:0E6AE000EF5C02E7DF0EEF16EE52F6E1120059
:026AEE00AA6A92
:106AF000A96A3F0EA6160B01B80E006F020E016FB9
:106B0000A950106E116A120E105C000E11580CE2A2
:106B1000A68000CBE9FF01CBEAFF002B000E01238A
:106B2000A8CFEFFFA92AECD71200D6C2A9FFAA6A04
:106B3000A6B2FED73F0EA616A680A8501200D7C256
:106B4000A9FFAA6AA6B2FED72F0EA616A684550ED6
:106B5000A76EAA0EA76EA6820000A6B2FED7A694C4
:106B600000D012001200240EAC6E900EAB6E080E18
:106B70007E6E02011F0E7CD8080A36E00F0A32E052
:106B8000010A2AE0030A23E0010A1CE0070A15E0D3
:106B9000010A0EE0030A07E0010A28E10B01340EA6
:106BA0001C6F820E1DD00B018C0E1C6F200E18D096
:106BB0000B01450E1C6F100E13D00B01220E1C6F23
:106BC000080E0ED00B01100E1C6F040E09D00B0125
:106BD000080E1C6F020E04D00B01030E1C6F010E79
:106BE0001D6F08D0AC0E03D0560E01D0AC0E0B01B9
:106BF0001C6F1D6B1CCBAFFF1DCB10F0116A10502A
:106C00007F6E12000201230E33D8926E0201240E11
:106C10002FD8936E0201250E2BD8D809946E02014D
:106C2000280E26D8976E0201290E22D81009986ED8
:106C3000120002012A0E1CD8896E02012B0E18D8F0
:106C40008A6E02012C0E14D88B6E02012F0E10D802
:106C50008E6E0201300E0CD88F6E12000201310EC2
:106C600007D8C16E0201320E03D87F0BC06E12002E
:066C7000D66F95EF35F030
:0A6C76000001EC6BE06BE16BEA6BD0
:106C8000EB6B9D9A9D9812009D8A9D9812000001C1
:106C9000E16BE1C0E0F0EB6BEBC0EAF01200060E36
:106CA000AB1402E0AB98AB889EAA0ED00001EB516A
:106CB000EA6AE20FE96E000EEA22AECFEFFFEB2B9D
:106CC000070EEB15EB6FF0D712000001E051E15D0C
:106CD0000DE0E051EA6A600FE96E000EEA22EF5023
:106CE000AD6EE02B7F0EE015E06F12009D98120054
:106CF00012000001EC5112000001EA51EA6AE20FB1
:106D0000E96E000EEA22EFCFAFFBEA2B070EEA1581
:106D1000EA6F0B01AF5112000001E129106E116AF8
:106D20007F0E1016000E11160001E051126E136A4C
:106D30001250101802E11350111802E10400ECD7B0
:106D4000F29E9DB805D0EDC0ADFF9D88F28E11D0AA
:106D50000001E151EA6A600FE96E000EEA22EDC01F
:106D6000EFFF0001E12B7F0E0001E1150001E16F53
:106D7000F28E12000001EE519F0805E2EE390F0B72
:106D80000F0B570F04D0EE390F0B0F0B300F000114
:106D9000ED6FC2DF0F0E0001EE15090804E20F0EC1
:106DA000EE15570F03D00F0EEE15300F0001ED6FEB
:106DB0008CEF36F00001EFC0E9FFF0C0EAFFEF2BE7
:106DC000000EF023EFCF08FBEF5004E008CBEDF00E
:106DD000A3DFF0D712000001F1C0F6FFF2C0F7FF09
:106DE000F12B000EF2230800F5CF00FBF55004E074
:0A6DF00000CBEDF091DFEFD71200A9
:066DFA000D01EF6BF069D2
:106E0000F169F269F369F469F569F66BF76BF86B90
:106E1000F96B12000D01EF5129E10301260E5D6FA0
:106E20000B0E5E6F03011C0E5B6F0B0E5C6F01ECB3
:106E30002DF000092CE00B01265115E11CCBF0FDD3
:106E40001DCBF1FD1ECBF2FD1FCBF3FD20CBF4FDDE
:106E500021CBF5FD22CBF6FD23CBF7FD24CBF8FDAE
:106E600025CBF9FD010C0D01010EEF6F34EC18F08C
:106E700000090CE00301616B03011C0E5F6F0B0E38
:106E8000606F74EC2DF00D01EF6B010C000C010C28
:106E9000FACDE9FFFBCDEAFFEECF22FBEECF23FBDD
:106EA000EECF24FBEFCF25FB0301010E616F030141
:106EB0001C0E5F6F0B0E606F74EF2DF0FCCDE9FFC1
:106EC000FDCDEAFF0D01F651EE1808E1F751EE187D
:106ED00005E1F851EE1802E1F951EE1814E0020153
:106EE000C6510D01F65D20E10201C7510D01F75DAC
:106EF0001BE10201C8510D01F85D16E10201C95103
:106F00000D01F95D11E1FECDE9FFFFCDEAFFF0CD06
:106F1000EEFFF1CDEEFFF2CDEEFFF3CDEEFFF4CDBF
:0A6F2000EEFFF5CDEEFF010C000CB2
:066F2A00545854004854C5
:106F30004D00434C4100435353004A53000047491E
:106F40004600434749004A5047004A4152005741D2
:106F50005600545854005A5458005A4854005A4342
:106F60004C005A4353005A4A5300485454502F314E
:106F70002E3020323030204F4B00436F6E74656EE0
:106F8000742D747970653A2000436F6E74656E7469
:106F90002D456E636F64696E673A20677A69700D7C
:106FA0000A00457870697265733A20300D0A004313
:106FB000616368652D436F6E74726F6C3A206D610A
:106FC000782D6167653D3330302C206D7573742DDD
:106FD000726576616C69646174650D0A0047455499
:106FE00000494E4445582E48544D004C4F47494E99
:056FF0002E434749009B
:0A6FF6002A0EF66E080EF76E000E6C
:10700000F86E02010900F550FB6F0900F550FC6FA6
:1070100003E1FB6701D03DD00900F550F66F090090
:10702000F550F76F0900F550F86F09000900F550A9
:10703000E96E0900F550EA6E090009000900F550F3
:10704000F96F0900F550FA6F09000900F6CFFDF25B
:10705000F7CFFEF2F8CFFFF2F6C2F6FFF7C2F7FF66
:10706000F8C2F8FF0201F95302E1FA5307E0090000
:10707000F550EE6EF907F8E2FA07F9D7FDC2F6FF10
:10708000FEC2F7FFFFC2F8FF0201FB07000EFC5B28
:04709000BFD7120054
:0C7094004E6F7420496D706C656D656E68
:1070A0007465640073656C6563746564006368652A
:1070B000636B65640064697361626C6564003C21A4
:1070C0002D2D002D2D3E006F6E006F6666005570F1
:0570D00064617465001D
:0A70D6003F0EC716C66AC56A030123
:1070E0007151C6127251C71294869488C68A73C3AE
:1070F000C8FF1200C586C7A0FED7C950120074C3CE
:0C710000C9FFC6BEFF0CC7B0FED7000CD4
:04710C00FF0EE3503F
:107110001D6EEF0E01D0F30EE76EE72E8DEF38F007
:107120000C0E1C6EE76AE72E93EF38F01C2E92EFE0
:0A71300038F01D2E8BEF38F012002E
:06713A00036A026A100E58
:10714000E76ED89006360736023603360B50025CDF
:107150000C50035805E30B50025E0C50035A062AEC
:06716000E72EF0D712003B
:0A7166000301646B656B666B676BD9
:10717000686B696B580ED66E9E0ED76E010ED56E7B
:08718000D58EF284F28A1200A0
:08718800036A080EE76ED890BF
:10719000073603360C50035C02E3036E072AE72E22
:0471A000F7D712000B
:0C71A4001EEE00F02EEE00F0F86A0F9CCA
:0C71B000FBEC37F0F0EC32F0FDD71200E1
:0471BC00FF0EE3508F
:1071C000E84E1200000000D000D000D0E82EFAD720
:0271D0001200AB
:0671D20056322E3433009A
:0671D80056332E30340096
:0271DE0019593D
:0E71E0000259E658CE58AE588D584E583158C8
:0271EE0000009F
:0271F00000009D
:0E71F20011580758F357EA57DA57D057075885
:10720000C557AC579F57115811580758F357EA57AD
:0A721000DA577857585753572C5798
:06721A00FC59F759F2597E
:10722000ED59E859E359D759BF59AF59A5599E5956
:0C7230008859735958594C5934592B593E
:04723C0000FF00004F
:020000040030CA
:0100010026D8
:0100020004F9
:010003000AF2
:010005008377
:010006008178
:010008000FE8
:010009008076
:01000A000FE6
:01000B008074
:01000C000FE4
:01000D0000F2
:0200000400F00A
:100000000A0100010004A3000000FF0000000A0133
:10001000000104012803000A0100010A0100010790
:10002000000700FFFFFFFFFFFFFF000000000000D0
:1000300000032E000061646D696E0000000070779F
:0700400000000000000000B9
:00000001FF
